:100000000C9473000C949B000C949B000C949B002C
:100010000C949B000C94891A0C949B000C949B00EC
:100020000C949B000C949B000C949B000C949B00E4
:100030000C949B000C949B000C949B000C949B00D4
:100040000C946E1E0C949B000C94FE0E0C94D80E17
:100050000C949B000C949B000C949B000C949B00B4
:100060000C94B60F0C949B004306450647064906C0
:100070004B064D064F0651068206850688067F060A
:100080008B068E06A006A0060000000025002800B2
:100090002B000000000023002600290004040404B3
:1000A0000404040402020202020203030303030322
:1000B00001020408102040800102040810200102FF
:1000C00004081020000000080002010000030407DB
:1000D00000000000000000000000000024002700D5
:1000E0002A007B2F4F2F11241FBECFEFD8E0DEBF99
:1000F000CDBF27E0A0EBB4E001C01D92AF30B20746
:10010000E1F714E0A0E0B1E0E0EFFEE602C0059008
:100110000D92A03BB107D9F710E0C2E7D0E004C0D0
:100120002197FE010E94C433C137D107C9F70E944D
:10013000B81E0C946B370C9400002F923F924F9294
:100140005F926F927F928F929F92AF92BF92CF9267
:10015000DF92EF92FF920F931F93CF93DF93CDB770
:10016000DEB768970FB6F894DEBF0FBECDBF522E34
:100170003D87442E5E873B011C01A982B98ACA8A49
:10018000DB8AEC8AFD8A0E8B1F8B988A8F8621155D
:1001900000EA30070CEA400709EB500703E060076C
:1001A00071058105910511F008F046C02F3F10EE52
:1001B000310715EF410715E051076105710581050C
:1001C000910561F058F02F3F354D41415E47634046
:1001D00071058105910509F0D8F50BC0512CF1EEA0
:1001E000FD87B5EF4B2E05E00E87612C712C212C7D
:1001F000312C298139894A895B896C897D898E896D
:100200009F89A0E00E94463509F0A7C0A52CBD84B7
:10021000C42CDE847301810120E034E04BE654EF0E
:1002200064E170E080E090E00E94903429873A8792
:100230004B875C87912C24C0512C10EA1D87FCEA67
:100240004F2E29EB2E87A3E06A2E712C212C312C06
:10025000298139894A895B896C897D898E899F8941
:10026000A0E00E94463509F0F4C09924939414E06C
:10027000E12EF12C00E010E0E986FA860B871C875E
:10028000E984FA840B851C85A801970160E070E081
:10029000CB01A52CBD84C42CDE847301810129838C
:1002A0003A834B835C836D837E838F83988760E082
:1002B00070E080E090E00E94CA332983398B4A8B3A
:1002C0005B8B6C8B7D8B8E8B9F8BFF24F3949F14A9
:1002D00009F4C2C010E0812C912C5401839440E0B9
:1002E00050E0BA0101C011E0CB01BA0107E0660F8E
:1002F000771F881F991F0A95D1F7C984DA84EB8488
:10030000FC8427E0CC0CDD1CEE1CFF1C2A95D1F7E9
:10031000A2E0DA1AE108F108A50194010E948333F2
:10032000C20ED31EE41EF51EEF85F889C082D1826D
:10033000E282F382648375838683978380869186C5
:10034000A286B3861111BBC0298139894A895B898C
:100350006C897D898E899F89B8C0188EA52CBD8433
:10036000C42CDE8473018101298139894A895B8922
:100370006C897D898E899F890E94903429873A876C
:100380004B875C8789859A85AB85BC850697A105D7
:10039000B10520F4B6E0AB2EB12C0FC0E984FA848D
:1003A0000B851C8529E0E21627E0F2060105110500
:1003B000D0F0F8E0AF2EA7E0BA2EC12CD12CE12C62
:1003C000F12C00E010E0298139894A895B896C8928
:1003D0007D898E899F890E949034522E3D87442EBC
:1003E0005E873B011C01A52CBD84C42CDE847301F7
:1003F0008101298139894A895B896C897D898E8946
:100400009F890E948E34AA24AA94BB24BA94EFE058
:10041000CE2ED12CE12CF12C00E010E00E94CA334A
:10042000A52CBD84C42CDE84730181010E9490340C
:10043000A32FF42FE52F422F5A2F6F2F7E2F411518
:10044000510561057105F9F4812C912C54018394B7
:1004500020C081E0888F82CFAF85B8891D921D9220
:100460001D921C921397FD01148215821682178229
:10047000C12CD12C7601C3941896CD92DD92ED92C9
:10048000FC921B9722C088248A94982C8FE0A82E77
:10049000B12CF88DF13009F026CFEF85F889108264
:1004A000118212821382148215821682178281E0D1
:1004B00090E0A0E0B0E080879187A287B387252DE8
:1004C0003D85442D5E85B301C10168960FB6F89451
:1004D000DEBF0FBECDBFDF91CF911F910F91FF9077
:1004E000EF90DF90CF90BF90AF909F908F907F90D4
:1004F0006F905F904F903F902F900895DF92EF9212
:10050000FF920F931F93CF93DF93FC01E080F18064
:1005100002811381D481C581B681D7809701A8015A
:100520006D2F7C2F8B2F9D2D35534C405109610928
:100530007109810991092F3F34434C4051056105F0
:1005400071058105910509F098F49701A8016D2FB7
:100550007C2F8B2F9D2D07E00E94FD34208331835B
:1005600042835383648375838683978387E0FDC0CA
:100570009701A8016D2F7C2F8B2F9D2D3A56484156
:10058000510961097109810991092F3F3946484193
:100590005105610571058105910509F098F49701F0
:1005A000A8016D2F7C2F8B2F9D2D06E00E94FD341E
:1005B0002083318342835383648375838683978347
:1005C00086E0D3C09701A8016D2F7C2F8B2F9D2D26
:1005D000345D4043510961097109810991092F3F37
:1005E000334D40435105610571058105910509F0C1
:1005F00098F49701A8016D2F7C2F8B2F9D2D05E07E
:100600000E94FD3420833183428353836483758346
:100610008683978385E0A9C09701A8016D2F7C2F61
:100620008B2F9D2D385A4146510961097109810965
:1006300091092F3F374A41465105610571058105F2
:10064000910509F098F49701A8016D2F7C2F8B2F4D
:100650009D2D04E00E94FD34208331834283538327
:10066000648375838683978384E07FC09701A801A4
:100670006D2F7C2F8B2F9D2D3055434C51096109D7
:100680007109810991092F3F3F44434C5105610590
:1006900071058105910509F098F49701A8016D2F66
:1006A0007C2F8B2F9D2D03E00E94FD34208331830E
:1006B00042835383648375838683978383E055C025
:1006C0009701A8016D2F7C2F8B2F9D2D305A464806
:1006D000514061097109810991092F3F3F494648FD
:1006E0005140610571058105910509F098F4970164
:1006F000A8016D2F7C2F8B2F9D2D02E00E94FD34D1
:1007000020833183428353836483758386839783F5
:1007100082E02BC09701A8016D2F7C2F8B2F9D2D80
:1007200030544D40534061097109810991092F3FAF
:100730003F434D405340610571058105910509F026
:1007400098F49701A8016D2F7C2F8B2F9D2D01E030
:100750000E94FD34208331834283538364837583F5
:100760008683978381E001C080E0DF91CF911F9164
:100770000F91FF90EF90DF900895CF93DF9391E07A
:1007800090939A0590E69093BC0510929B05109269
:10079000BD05682F8BE596E00E94C70D81E00E94A1
:1007A000051D809199058111FCCF81E08093990509
:1007B000109298059FEF90939705109296051092CE
:1007C00095058093740580917405806C8093740501
:1007D00080917305813061F41092730580917405E6
:1007E0008093BB008091BC0083FDF8CF85EC01C0F5
:1007F00085EE8093BC00809199058130E1F3809172
:100800009605811103C0C091960501C0C1E0E5E7DE
:10081000F5E0ACE0B5E080E08C1721F091919D937C
:100820008F5FFACF10920B05C0930A0580910B05DC
:10083000C81731F08BE596E00E947E0DD82FF6CFD9
:100840008D2FDF91CF9108952F923F924F925F921B
:100850006F927F928F929F92AF92BF92CF92DF92D0
:10086000EF92FF920F931F93CF93DF93CDB7DEB735
:1008700061970FB6F894DEBF0FBECDBF2D833E83C8
:100880004F83588769877A871C011F870E8760917D
:10089000E6067091E7068091E8069091E90624E665
:1008A00030E040E050E00E9432342D87388B4B8797
:1008B0005C87762E672E582E492E8091E006909107
:1008C000E106A091E206B091E3066C017D01FF0C08
:1008D000CC08DC2C76019C01AD016C2D7C2D8C2D7F
:1008E0009C2D0FE10E94FD34A12C0AECB02EEAE908
:1008F000CE2EFBE3DF2EE12CF12C00E010E00E9475
:100900005F34AD84B888CB84DC84E72CF62C052DCD
:10091000142D0E94CA330FE10E94183549015A0173
:10092000D501C401BB0F880B982FDC0189839A8302
:10093000AB83BC839401A5016981762F862F962F06
:10094000AD84B888CB84DC84E72CF62C052D0E947E
:1009500034352983832E942E598B688B7B878C8723
:100960009D872D813E814F81588569857A85C1019A
:100970002F3FA7E53A07A7E44A07A8EF5A07ADE0DB
:100980006A07710581059105A9F0A0F02115344091
:100990004B46544F6441710581059105B9F0B0F0A3
:1009A0001D8294E09E83ABE6AF83B4EFB887E4E1A9
:1009B000E98709C01D82E8E5EE83F7E4FF8328EFAD
:1009C00028878DE089871A86212C312CA980B82CA4
:1009D000C92CD988E888FB840C851D852D813E8132
:1009E0004F81588569857A85C1010E94903429011B
:1009F0003A01FFE04F1651046104710418F4AFE0AE
:100A0000AA2E08C02BE54216510461047104D0F0EF
:100A1000FAE5AF2EB12CC12CD12CE12CF12C00E049
:100A200010E02981382D492D598968897B858C856D
:100A30009D850E94CA332D833E834F8358876987E3
:100A40007A871C01A980B82CC92CD988E888FB8436
:100A50000C851D852D813E814F81588569857A855C
:100A6000C1010E948E34AA24AA94BB24BA94EFE058
:100A7000CE2ED12CE12CF12C00E010E00E94CA33E4
:100A8000A980B82CC92CD988E888FB840C851D85E1
:100A90000E949034C901DA010097A105B10529F43B
:100AA000C12CD12C7601C39406C0CC24CA94DC2C72
:100AB0005FE0E52EF12CBC01CD0127E0660F771F2A
:100AC000881F991F2A95D1F737E0440C551C661CE6
:100AD000771C3A95D1F7A2E05A1A61087108A7016C
:100AE00096010E948333862E372E982E420E531E77
:100AF000641E751E84E190E00E9466359A838983A6
:100B0000FC01D082C182862D83708283538244820D
:100B1000D701C6014CE0B695A795979587954A955C
:100B2000D1F7807FC82EC90CC582368287828E8518
:100B30009F85892B19F4BF018AE107C0AE85BF8567
:100B4000119729F469817A8182E20E94611D89816D
:100B50009A8161960FB6F894DEBF0FBECDBFDF91CC
:100B6000CF911F910F91FF90EF90DF90CF90BF90AA
:100B7000AF909F908F907F906F905F904F903F903D
:100B80002F900C94FE35CF93C62F91E090939A0549
:100B900090E69093BC0510929B051092BD05682FBE
:100BA0008BE596E00E94C70D6C2F8BE596E00E94C6
:100BB000C70D81E0CF910C94051D2F923F924F926B
:100BC0005F926F927F928F929F92AF92BF92CF92DD
:100BD000DF92EF92FF920F931F93CF93DF93CDB7E6
:100BE000DEB72E970FB6F894DEBF0FBECDBF3C0127
:100BF000C982DA82EB82FC820D831E832F833887C1
:100C000049875A876B877C878BA18D873C2C2D2C3D
:100C10005E2C0E87412E922EC984DA84EB84FC84EC
:100C200084E190E00E9466358C01FC01D082C18293
:100C3000862D880F880F880F845D0E94BD03952D37
:100C400093708C7F892BF801828323823482D701B1
:100C5000C6017CE0B695A795979587957A95D1F7CB
:100C6000807F992D9F70C92EC80EC58246828E85C1
:100C7000878398E069167104B8F4F301EC5CFF4FC8
:100C8000B8010C94C4338AE20DC082E30BC08AE33E
:100C900009C082E407C08AE405C082E503C08AE592
:100CA00001C08BE50E94611D60E1F62EF60C8F2DD0
:100CB0000E94BD03E1E0682FAE1202C0606401C073
:100CC0006F7B8F2D0E94C305F1E06F16710459F000
:100CD00038F092E06916710449F4A092DF0618C05A
:100CE000A092DD060FC0A092DE060FC0E8E06E16EF
:100CF0007104B0F4F301E45CFF4F0C94C43354E48A
:100D0000B52E0EC04CE2B42E0BC034E3B32E08C097
:100D10002CE3B22E05C09CE4B92E02C084E5B82EA7
:100D20008B2D0E94BD038378FD85F1118C6090E1CD
:100D3000899E40011124682F68298B2D0E94C305CC
:100D4000C8012E960FB6F894DEBF0FBECDBFDF915F
:100D5000CF911F910F91FF90EF90DF90CF90BF90B8
:100D6000AF909F908F907F906F905F904F903F904B
:100D70002F900C94FE350F931F93CF938B01C0E1FE
:100D8000C80F8C2F0E94BD030115110511F48F7D32
:100D900004C00130110509F48062682F8C2FCF91B7
:100DA0001F910F910C94C3052F923F924F925F9227
:100DB0006F927F928F929F92AF92BF92CF92DF926B
:100DC000EF92FF920F931F93CF93DF93CDB7DEB7D0
:100DD000AA970FB6F894DEBF0FBECDBF622E298F43
:100DE000732E3A8F4B8F5C8F6D8F7E8F8F8F98A372
:100DF00019A708A793012F3F34434C4051056105C3
:100E000071058105910509F050F4198E85E38A8FEB
:100E10008CE08B8F1C8E1D8E1E8E1F8E18A2298D2E
:100E20003A8D4B8D5C8D6D8D7E8D8F8D98A12115AA
:100E3000304A4C4A594B634071058105910569F070
:100E400060F0198E80EA8A8F8CEA8B8F89EB8C8F09
:100E500083E08D8F1E8E1F8E18A2CE0149960E94B0
:100E60007E028AA7798CBA8DAB8DFC8DED8D6E8C50
:100E70005F8C48A0272D3B2F4A2F5F2F6E2F762D9A
:100E8000852D942D2F3F05ED300701E140070EE73A
:100E9000500703E0600771058105910511F008F026
:100EA0007FC09E01235F3F4F4901A12CEEE2BE2E81
:100EB000F9E5CF2EA6E7DA2E11E1E12EF12C00E0C4
:100EC00010E0272D3B2F0E949D0088A599A5813019
:100ED000910509F44CC038F1029709F065C3898D7A
:100EE0008093D5068A8D8093D6068B8D8093D70606
:100EF0008C8D8093D8068D8D8093D9068E8D8093AE
:100F0000DA068F8D8093DB0688A18093DC0680E073
:100F100019A2212C3EE2332E49E5442E16E71CA3EC
:100F200021E12DA34CC3898D8093C5068A8D8093C2
:100F3000C6068B8D8093C7068C8D8093C8068D8DD9
:100F40008093C9068E8D8093CA068F8D8093CB06C1
:100F500088A18093CC0680E019A2212C5EE2352E78
:100F600069E5462E96E79CA3E1E1EDA328C3898DB0
:100F70008093CD068A8D8093CE068B8D8093CF068D
:100F80008C8D8093D0068D8D8093D1068E8D80932D
:100F9000D2068F8D8093D30688A18093D40604C394
:100FA000CE010D964C01A12CB12CC12CD12CE12CE1
:100FB000F12C00E010E0272D3B2F4A2F5F2F6E2FE2
:100FC000762D852D942D0E949D00E8A5F9A5E13090
:100FD000F10509F458C020F0329709F49AC115C3FD
:100FE000298D3A8D4B8D5C8D6D8D7E8D8E01035FCD
:100FF0001F4F4801A12CB12CC12CD12CE12CF12C7C
:1010000000E010E08F8D98A10E949D001901442EF0
:101010005CA36DA3772E582E692E60E070E080E00F
:1010200090E00E94BB062092B5063092B606409230
:10103000B7061CA11093B8062DA12093B906709293
:10104000BA065092BB066092BC06898D8093C50695
:101050008A8D8093C6068B8D8093C7068C8D809376
:10106000C8068D8D8093C9068E8D8093CA068F8D9C
:101070008093CB0688A18093CC0681E031E039A330
:101080001BA21AA29FC21091E506B98DAA8DFB8DF5
:10109000EC8D0D8D09A30E8D0AA30F8D0EA308A153
:1010A0000FA3123009F073C02B2F3A2F4F2F5E2F52
:1010B00069A17AA18EA1902F30584A41564061090A
:1010C0007109810991092F37304E424758496240D2
:1010D00071058105910569F160F1A090D506B09088
:1010E000D606C090D706D090D806E090D906F090EA
:1010F000DA060091DB061091DC062B2F3A2F4F2FDA
:101100005E2F69A17AA18EA19FA10E943D3589F031
:101110001092CD061092CE061092CF061092D006F5
:101120001092D1061092D2061092D3061092D406D5
:101130006CC22090BD063090BE064090BF06209144
:10114000C0062CA33091C1063DA37090C2065090FA
:10115000C3066090C406CE010D964C015101C42C0B
:10116000D22EE32EF72C052D162D2B2F3A2F4F2F95
:101170005E2F69A17AA18EA19FA10E949D0061E0CE
:1011800070E081E090E00E94BB0619A235C0209378
:10119000BD063093BE064093BF065093C0066093D1
:1011A000C1067093C2068093C3069093C4068E0155
:1011B000035F1F4F4801A12CB12CC12CD12CE12C75
:1011C000F12C00E010E02B2F3A2F4F2F5E2F69A15A
:1011D0007AA18EA19FA10E949D001901442E5CA3BB
:1011E0006DA3772E582E692E61E070E081E090E0CB
:1011F0000E94BB0611E019A3298D3A8D4B8D5C8DA1
:101200006D8D7E8D8F8D98A130584A415640610971
:101210007109810991092F37304E42475849624080
:1012200071058105910509F008F457C081E08093AC
:10123000E5062091D5063091D6064091D70650910B
:10124000D8066091D9067091DA068091DB069091FC
:10125000DC06A0E00E94463509F442C085ED96E028
:101260000E947E028AA7A090BD06B090BE06C090E4
:10127000BF06D090C006E090C106F090C206009173
:10128000C3061091C4062091D5063091D606409130
:10129000D7065091D8066091D9067091DA06CE0132
:1012A00001964C018091DB069091DC060E949D0026
:1012B0001F928AA4A12CC980DA80EB80FC800D816A
:1012C0001E812F81388549855A856B857C8582E012
:1012D00090E00E94DD050F9003C088E08093E50652
:1012E000898D8093CD068A8D8093CE068B8D8093D9
:1012F000CF068C8D8093D0068D8D8093D1068E8DF8
:101300008093D2068F8D8093D30688A18093D406D4
:1013100045C17090E506B98DAA8DFB8DEC8D0D8DC4
:1013200009A31E8D1AA30F8D0EA318A11FA301E000
:10133000701273C02B2F3A2F4F2F5E2F69A17AA105
:101340008EA1912F30584A41564061097109810997
:1013500091092F37304E4247584962407105810547
:10136000910569F160F1A090D506B090D606C090C5
:10137000D706D090D806E090D906F090DA06009112
:10138000DB061091DC062B2F3A2F4F2F5E2F69A121
:101390007AA18EA19FA10E943D3589F01092D506B9
:1013A0001092D6061092D7061092D8061092D9063F
:1013B0001092DA061092DB061092DC062AC1209009
:1013C000BD063090BE064090BF062091C0062CA3FB
:1013D0003091C1063DA37090C2065090C306609044
:1013E000C406CE010D964C015101C42CD22EE32E21
:1013F000F72C052D162D2B2F3A2F4F2F5E2F69A17D
:101400007AA18EA19FA10E949D0061E070E082E020
:1014100090E00E94BB0619A235C02093BD06309310
:10142000BE064093BF065093C0066093C1067093FA
:10143000C2068093C3069093C4068E01035F1F4FBC
:101440004801A12CB12CC12CD12CE12CF12C00E0B5
:1014500010E02B2F3A2F4F2F5E2F69A17AA18EA17A
:101460009FA10E949D001901442E5CA36DA3772EBD
:10147000582E692E61E070E082E090E00E94BB0689
:1014800011E019A3298D3A8D4B8D5C8D6D8D7E8D6C
:101490008F8D98A130584A415640610971098109E0
:1014A00091092F37304E42475849624071058105F6
:1014B000910509F008F457C082E08093E506209179
:1014C000CD063091CE064091CF065091D006609166
:1014D000D1067091D2068091D3069091D406A0E0F7
:1014E0000E94463509F442C08DEC96E00E947E02CF
:1014F0008AA7A090BD06B090BE06C090BF06D0904F
:10150000C006E090C106F090C2060091C30610919B
:10151000C4062091CD063091CE064091CF06509161
:10152000D0066091D1067091D206CE0101964C0191
:101530008091D3069091D4060E949D001F928AA4A8
:10154000A12CC980DA80EB80FC800D811E812F8167
:10155000388549855A856B857C8581E090E00E94BD
:10156000DD050F9003C088E08093E506898D8093A8
:10157000D5068A8D8093D6068B8D8093D7068C8D69
:101580008093D8068D8D8093D9068E8D8093DA0650
:101590008F8D8093DB0688A18093DC0681E0E1E0FB
:1015A000F0E0FBA3EAA30EC080E019A2212C9EE28A
:1015B000392E29E5422EF6E7FCA301E10DA3712C9B
:1015C000512C612C8F938AA4A82ECD84DE84EF84C5
:1015D000F88809891A892B893C894D895E896F8928
:1015E000788D88A599A50E94DD050F9019A111306D
:1015F00079F40AA11BA19101442D5CA16DA1772D65
:10160000852D962D0E94240403C07724739401C075
:10161000712C872DAA960FB6F894DEBF0FBECDBFF2
:10162000DF91CF911F910F91FF90EF90DF90CF90BE
:10163000BF90AF909F908F907F906F905F904F90F2
:101640003F902F9008951F93CF93DF93EC01162FB7
:1016500083E00E94BD039E01332761E070E001C07A
:10166000660F2A95EAF7113019F46095682301C0D6
:10167000682B83E0DF91CF911F910C94C3050097F5
:1016800069F0FC0101900020E9F73197AF01481B98
:10169000590BBC0185E896E00C94380E80E0089563
:1016A000CF92DF92EF92FF92CF93DF9397FF19C013
:1016B0006B017C018DE20E94ED1BEC016627772710
:1016C000CB016C197D098E099F094AE00E94F61B27
:1016D0008C0F9D1FDF91CF91FF90EF90DF90CF9007
:1016E00008954AE0DF91CF91FF90EF90DF90CF9087
:1016F0000C94F61BCF93C0E1C80F8C2F0E94BD0342
:10170000682F63608C2FCF910C94C3050F931F93A8
:10171000CF93DF938B01877028E0829FC001112453
:1017200080640E942D1BE801085F1F4F69918AEEBB
:1017300096E00E94B00FC017D107C1F7DF91CF919B
:101740001F910F910895CF93DF93282F30E0F90177
:10175000EC53FF4F8491F901E055FF4FD491F9010B
:10176000E456FF4FC491CC2391F081110E94AC1D2F
:10177000EC2FF0E0EE0FFF1FEE56FF4FA591B49156
:10178000EC91ED2381E090E021F480E002C080E064
:1017900090E0DF91CF9108951F93CF93DF93282F8F
:1017A00030E0F901EC53FF4F8491F901E055FF4F10
:1017B000D491F901E456FF4FC491CC23C1F0162F08
:1017C00081110E94AC1DEC2FF0E0EE0FFF1FE857D7
:1017D000FF4FA591B4919FB7F894111104C08C915B
:1017E000D095D82302C0EC91DE2BDC939FBFDF9114
:1017F000CF911F91089510920B0510920A05109237
:101800009B051092BD051092990581E08093980583
:101810001092730561E082E10E94CC0B61E083E1EC
:101820000E94CC0BE9EBF0E080818E7F8083808189
:101830008D7F808388E48093B80085E48093BC002A
:101840008CE69DE090930905809308058DE69DE068
:10185000909307058093060508950895CF92DF922F
:10186000EF92FF920F931F93CF93DF936C017A0156
:101870008B01C0E0D0E0CE15DF0581F0D8016D917D
:101880008D01D601ED91FC910190F081E02DC60112
:101890000995892B11F02196EECF7E01C701DF91CA
:1018A000CF911F910F91FF90EF90DF90CF9008950F
:1018B000FC01538D448D252F30E0842F90E0821B56
:1018C000930B541710F0CF96089501970895FC01DB
:1018D000918D828D981761F0828DDF01A80FB11D67
:1018E0005D968C91928D9F5F9F73928F90E008958B
:1018F0008FEF9FEF0895FC01918D828D981731F045
:10190000828DE80FF11D858D90E008958FEF9FEF98
:101910000895FC01918D228D892F90E0805C9F4F6E
:10192000821B91098F73992708958EEB95E00E9491
:10193000890C21E0892B09F420E0822F0895FC0115
:10194000848DDF01A80FB11DA35ABF4F2C91848D48
:1019500090E001968F739927848FA689B7892C937D
:10196000A089B1898C91837080648C93938D848DD0
:10197000981306C00288F389E02D80818F7D8083D3
:101980000895EF92FF920F931F93CF93DF93EC0193
:1019900081E0888F9B8D8C8D981305C0E889F9892B
:1019A000808185FD26C0F62E0B8D10E00F5F1F4F46
:1019B0000F731127E02E8C8DE8120CC00FB607FCB8
:1019C000FACFE889F989808185FFF5CFCE010E94A1
:1019D0009F0CF1CF8B8DFE01E80FF11DE35AFF4FF5
:1019E000F0829FB7F8940B8FEA89FB89808180622F
:1019F0000AC09FB7F894EE89FF896083E889F98966
:101A000080818370806480839FBF81E090E0DF915C
:101A1000CF911F910F91FF90EF900895CF93DF9397
:101A2000EC01888D8823C9F0EA89FB89808185FDD6
:101A300005C0A889B9898C9186FD0FC00FB607FC37
:101A4000F5CF808185FFF2CFA889B9898C9185FF78
:101A5000EDCFCE010E949F0CE7CFDF91CF9108958B
:101A600080E090E0892B29F00E94950C81110C9464
:101A70000000089585ED8093BC008091BC0084FD3A
:101A8000FCCF10929905089540915005262F30E023
:101A9000240F311D21323105DCF4209199052430C9
:101AA000C9F4FC0180E090E0861758F430915005AD
:101AB0002191DC01A05DBA4FA30FB11D2C930196BB
:101AC000F3CF80915005680F6093500580E0089532
:101AD00081E0089582E00895089508950895E091C1
:101AE0000B0580910A05E81730F4F0E0E45FFA4F47
:101AF000808190E008958FEF9FEF089590910B05FE
:101B000080910A05981750F4E92FF0E0E45FFA4F4E
:101B1000208130E09F5F90930B0502C02FEF3FEFD5
:101B2000C901089580910A0590E020910B05821B60
:101B300091090895CF92DF92EF92FF920F931F9336
:101B4000CF93DF937C01CB018A0120919A05222358
:101B500089F0EB016B01C40ED51ECC15DD0569F0D3
:101B60006991D701ED91FC910190F081E02DC701C1
:101B70000995F3CF642F0E94440DC801DF91CF91E6
:101B80001F910F91FF90EF90DF90CF900895CF932A
:101B9000DF931F92CDB7DEB7698320919A05222388
:101BA000D1F02091BD05203240F021E030E0FC0171
:101BB0003383228380E090E015C080919B05E82F5D
:101BC000F0E0E456FA4F998190838F5F80939B05F4
:101BD0008093BD0505C061E0CE0101960E94440DD1
:101BE00081E090E00F90DF91CF91089580E090E048
:101BF00008950E944D370F931F93CF93DF93EC010D
:101C000088819981009729F02A813B81261737071F
:101C100088F48B016F5F7F4F0E948736009761F0D9
:101C2000998388831B830A832C813D81232B11F4A4
:101C3000FC01108281E001C080E0DF91CF911F9113
:101C40000F910895CF93DF93EC0160E08E810E94A5
:101C5000CC0B61E08E810E94CC0B60E08E810E94F3
:101C6000CC0B8BE891E00197F1F7DF91CF910895CC
:101C7000EF92FF920F931F93CF93DF93611571053E
:101C800011F480E01CC041155105C1F07B01EC014D
:101C90008C819D818A01080F191FB801CE010E9415
:101CA000FB0D882371F3288139818C819D81B701D7
:101CB000820F931F0E9464371D830C8381E0DF91A4
:101CC000CF911F910F91FF90EF900895CF93DF93E5
:101CD000EC0188819981009711F00E94FE351982EC
:101CE00018821D821C821B821A82DF91CF91089577
:101CF000EF92FF920F931F93CF93DF93EC017B0141
:101D00008A01BA010E94FB0D811104C0CE010E941C
:101D1000660E07C01D830C83B701888199810E94DC
:101D20006437CE01DF91CF911F910F91FF90EF901B
:101D30000895CF93DF93EC016115710559F0FB0114
:101D400001900020E9F73197AF01461B570B0E9425
:101D5000780E02C00E94660ECE01DF91CF910895E9
:101D6000FC01808191810C94FE35FC01118210826E
:101D700013821282158214826115710551F0FB01E4
:101D800001900020E9F73197AF01461B570B0C94E7
:101D9000780E0895DB0114964D915C9115976D9125
:101DA0007C91DC01ED91FC910280F381E02D09949E
:101DB0001F920F920FB60F9211242F933F934F93C0
:101DC0005F936F937F938F939F93AF93BF93EF93A3
:101DD000FF938EEB95E00E949F0CFF91EF91BF91D6
:101DE000AF919F918F917F916F915F914F913F91B3
:101DF0002F910F900FBE0F901F9018951F920F926A
:101E00000FB60F9211242F938F939F93EF93FF930D
:101E1000E091CE05F091CF058081E091D405F0915D
:101E2000D50582FD12C090818091D7058F5F8F7399
:101E30002091D805821751F0E091D705F0E0E254E7
:101E4000FA4F958F8093D70501C08081FF91EF9164
:101E50009F918F912F910F900FBE0F901F9018950B
:101E6000CF92DF92EF92FF920F931F93CF93DF9366
:101E70006C017C0187E0E80EF11CC0E0D0E0062F89
:101E800010E0B8010C2E02C0759567950A94E2F730
:101E90006170F70181917F010E94CC0B2196C430C3
:101EA000D10579F7C601DF91CF911F910F91FF9076
:101EB000EF90DF90CF900C94220ECF92DF92EF92B2
:101EC000FF920F931F93CF93DF93EC01F62E642FB5
:101ED0008C810E94CC0B8D818F3F19F060E00E94B5
:101EE000CC0B8F850F2D10E084FF25C06E0187E09D
:101EF000C80ED11CE12CF12CB8010E2C02C0759536
:101F000067950A94E2F76170F60181916F010E9472
:101F1000CC0BFFEFEF1AFF0A88E0E816F10461F737
:101F2000CE01DF91CF911F910F91FF90EF90DF9045
:101F3000CF900C94220EB80184E0759567958A9530
:101F4000E1F7CE010E94300F6F2DCE01DF91CF91CE
:101F50001F910F91FF90EF90DF90CF900C94300F76
:101F600041E00E945D0F81E090E008951F920F9282
:101F70000FB60F9211242F933F934F935F936F935C
:101F80007F938F939F93AF93BF93EF93FF93809132
:101F9000B900887F803609F49CC068F5883209F45E
:101FA0005BC090F4803109F454C038F4882309F4FC
:101FB000F6C0883009F44DC0F6C0883109F44CC031
:101FC000803209F45DC0EFC0803409F468C048F481
:101FD000803309F455C0883309F0E5C08093970534
:101FE000D8C0803509F44FC0883509F45DC0883405
:101FF00009F0D9C0D6C0883909F4C7C0A8F4883719
:1020000009F467C038F4883609F463C0803709F4EE
:1020100060C0C9C0883809F4B8C0803909F45FC00D
:10202000803809F0C0C05BC0803B09F486C038F43A
:10203000803A09F466C0883A09F47FC0B4C0803C95
:1020400009F4A7C0883C09F4A4C0883B09F48AC0FD
:10205000AAC08091740510C0909196058091950555
:10206000981770F5E091960581E08E0F80939605A4
:10207000F0E0EB58FA4F80818093BB0085EC86C07E
:10208000809397058EC0E091960581E08E0F809336
:1020900096058091BB00F0E0EB58FA4F8083909159
:1020A0009605809195056EC0E091960581E08E0FB2
:1020B000809396058091BB00F0E0EB58FA4F808347
:1020C0008091980581116DC081E08093730584EA49
:1020D00061C083E08093990510927205CFCF809103
:1020E0007205803208F051C0E091720581E08E0FD8
:1020F000809372058091BB00F0E0EE5AFA4F808326
:10210000BDCF85EC8093BC0010929905809172053B
:10211000803230F4E0917205F0E0EE5AFA4F10820E
:102120006091720570E0E0910605F091070582E587
:1021300095E009951092720536C084E08093990568
:102140001092510510925005E0910805F091090593
:10215000099580915005811105C081E0809350055B
:1021600010923005E091510581E08E0F809351056A
:10217000F0E0E05DFA4F80818093BB0090915105C3
:1021800080915005981708F479CF85E88093BC00BA
:102190000AC085EC8093BC001092990504C010928F
:1021A00097050E943A0DFF91EF91BF91AF919F91DA
:1021B0008F917F916F915F914F913F912F910F90F0
:1021C0000FBE0F901F9018950F931F93CF93DF931F
:1021D0008C01EB010E94E0318883C80101960E94C6
:1021E000E0318983CE01DF91CF911F910F91089546
:1021F000CF92DF92EF92FF920F931F93CF93DF93D3
:10220000EB017B0124E0E20EF11C8B016C01C61A8C
:10221000D70AC601800F911F0E94E031F801819317
:102220008F01EE15FF05A9F7CE01DF91CF911F9128
:102230000F91FF90EF90DF90CF900895AF92BF92F3
:10224000CF92DF92EF92FF920F931F93CF93DF9382
:1022500000D0CDB7DEB78B016B0124E0C20ED11CDC
:102260007B015C01A61AB70AC5018E0D9F1DF701FF
:1022700061917F019A838983CE0101960E94021B9E
:10228000EC14FD0489F7C8010F900F90DF91CF91F6
:102290001F910F91FF90EF90DF90CF90BF90AF9084
:1022A0000895EF92FF920F931F93CF93DF9300D087
:1022B000CDB7DEB78C017B01FB0160819A838983F6
:1022C000CE0101960E94021BF70161810F5F1F4F33
:1022D0001A830983CE0101960E94021BC7010F9049
:1022E0000F90DF91CF911F910F91FF90EF90089584
:1022F0000F931F93CF93DF9300D0CDB7DEB78B0141
:10230000FB0160819A838983CE0101960E94021BA2
:10231000C8010F900F90DF91CF911F910F910895F9
:10232000CF93DF93EB010E94E0318883CE01DF91F0
:10233000CF9108958091BD049091BE04A091BF04F7
:10234000B091C0040A97A105B1051CF480E20E9477
:10235000ED1B80E20E94ED1B6091BD047091BE04F4
:102360008091BF049091C0040E94500B8EE20E94A5
:10237000ED1B6091C1047091C2048091C3049091DF
:10238000C40420E432E44FE050E00E94A53328EE7C
:1023900033E040E050E00E94A5332093BD04309329
:1023A000BE044093BF045093C00424363105410558
:1023B00051051CF480E30E94ED1B8091BD049091B7
:1023C000BE04A091BF04B091C0040A97A105B10555
:1023D0001CF480E30E94ED1B6091BD047091BE046B
:1023E0008091BF049091C0040E94500B8EE20E9425
:1023F000ED1B6091C1047091C2048091C30490915F
:10240000C40428EE33E040E050E00E94A53360931E
:10241000BD047093BE048093BF049093C0046436DF
:102420007105810591051CF480E30E94ED1B8091EC
:10243000BD049091BE04A091BF04B091C0040A975E
:10244000A105B1051CF480E30E94ED1B6091BD0461
:102450007091BE048091BF049091C0040C94500B05
:102460008FE00E94111E9093CA048093C904BC019E
:10247000990F880B990B0E94C33020E030E040EAAE
:1024800050E40E94223120E030E040E85AE30E940C
:10249000223160932C0570932D0580932E05909327
:1024A0002F0508950F931F930E94621E0091CB0485
:1024B0001091CC042091CD043091CE04DC01CB01ED
:1024C000801B910BA20BB30B853F9140A105B10579
:1024D00008F4DEC161E080E00E94DB1B83EF93E043
:1024E0000E94D91B60912C0570912D0580912E05BD
:1024F00090912F0542E00E94371C84E694E00E94F0
:10250000D91B8091B8048130C1F40E94301260E080
:1025100080E00E94DB1B8FEF93E00E94D91B80912B
:10252000C9049091CA04909327018093260166E222
:1025300071E084E690E00E9451118091B8048230ED
:10254000D1F50E94301260E080E00E94DB1B81E147
:1025500094E00E94D91B8091C9049091CA04909381
:102560007201809371012091260130912701821B15
:10257000930B63E070E00E946F33260F371F309398
:10258000250120932401260F371F309370012093DB
:102590006F0164E271E087E690E00E9451116FE6FE
:1025A00071E08AE690E00E94511161E771E08DE6EA
:1025B00090E00E9451118091B8048330D1F50E94BF
:1025C000301260E080E00E94DB1B82E294E00E9417
:1025D000D91B8091C9049091CA049093780180938B
:1025E00077012091710130917201821B930B63E09E
:1025F00070E00E946F33260F371F309374012093D1
:102600007301260F371F309376012093750163E71E
:1026100071E080E790E00E94511165E771E083E787
:1026200090E00E94511167E771E086E790E00E9418
:1026300051118091B8048430D1F50E94301260E0CD
:1026400080E00E94DB1B83E394E00E94D91B809111
:10265000C9049091CA0490937E0180937D012091DA
:10266000770130917801821B930B63E070E00E9448
:102670006F33260F371F30937A0120937901260F8D
:10268000371F30937C0120937B0169E771E089E774
:1026900090E00E9451116BE771E08CE790E00E949E
:1026A00051116DE771E08FE790E00E945111809128
:1026B000B804853009F048C00E94301260E080E024
:1026C0000E94DB1B84E494E00E94D91B8091C90422
:1026D0009091CA04909386018093850120917D0199
:1026E00030917E01821B930B97FD039695958795FC
:1026F00095958795280F391F3093800120937F018E
:10270000280F391F3093820120938101820F931F7C
:1027100090938401809383016FE771E082E890E0F9
:102720000E94511161E871E085E890E00E9451112A
:1027300063E871E088E890E00E94511165E871E07B
:102740008BE890E00E9451118091B804863009F026
:1027500048C00E94301260E080E00E94DB1B85E5EB
:1027600094E00E94D91B8091C9049091CA0490936F
:102770008E0180938D012091850130918601821B0D
:10278000930B97FD03969595879595958795280FBB
:10279000391F3093880120938701280F391F309308
:1027A0008A0120938901820F931F90938C0180935B
:1027B0008B0167E871E08EE890E00E94511169E8B2
:1027C00071E081E990E00E9451116BE871E084E9C9
:1027D00090E00E9451116DE871E087E990E00E945D
:1027E00051118091B804873009F048C00E9430121E
:1027F00060E080E00E94DB1B86E694E00E94D91B2B
:102800008091C9049091CA04909396018093950198
:1028100020918D0130918E01821B930B97FD0396C1
:102820009595879595958795280F391F3093900139
:1028300020938F01280F391F30939201209391012B
:10284000820F931F90939401809393016FE871E03E
:102850008AE990E00E94511161E971E08DE990E010
:102860000E94511163E971E080EA90E00E945111E9
:1028700065E971E083EA90E00E9451110E94621EB6
:102880006093CB047093CC048093CD049093CE04DA
:102890001F910F9108958F929F92AF92BF92FF92D6
:1028A0000F931F93CF93DF93EC01F090D704009127
:1028B000D8041091D904F110A0C00230110509F418
:1028C0009CC08130910509F04BC08091B8048F5FA6
:1028D000873008F087E08093B804409165015091FB
:1028E000660160916701709168018091A8019091E3
:1028F000A901A091AA01B091AB01840F951FA61F59
:10290000B71F8093A8019093A901A093AA01B09347
:10291000AB016091A8017091A9018091AA019091E9
:10292000AB012091650130916601409167015091A2
:1029300068018090650190906601A0906701B09059
:1029400068010E948333C501B4010E945F33609324
:10295000A8017093A9018093AA019093AB014DC087
:10296000019609F04AC0409165015091660160915D
:102970006701709168018091A8019091A901A091CF
:10298000AA01B091AB01841B950BA60BB70B8093EA
:10299000A8019093A901A093AA01B093AB01609103
:1029A000A8017091A9018091AA019091AB01209199
:1029B00065013091660140916701509168018090F6
:1029C000650190906601A0906701B09068010E9437
:1029D0008333C501B4010E945F336093A8017093F3
:1029E000A9018093AA019093AB018091B804815012
:1029F000823008F481E08093B8048091A80190911E
:102A0000A901A091AA01B091AB018130914EA54FCF
:102A1000B54060F080E091EEA5EFB5E08093A801AD
:102A20009093A901A093AA01B093AB018091A80152
:102A30009091A901A091AA01B091AB018032914A75
:102A4000A740B10560F480E291EAA7E0B0E080938E
:102A5000A8019093A901A093AA01B093AB0121E032
:102A6000F2129AC0C130D10509F045C080916501CC
:102A700090916601A0916701B09168014091C504F1
:102A80005091C6046091C7047091C804840F951FCB
:102A9000A61FB71F8093C5049093C604A093C704D4
:102AA000B093C8040130110509F087C08091D304A8
:102AB0009091D404A091D504B091D6048093A8013C
:102AC0009093A901A093AA01B093AB0180916501F5
:102AD00090916601A0916701B091680140916B01EE
:102AE00050916C0160916D0170916E01840F951F82
:102AF000A61FB71F48C0CF3F8FEFD80709F0EFC21E
:102B00004091650150916601609167017091680183
:102B10008091C5049091C604A091C704B091C804E7
:102B2000841B950BA60BB70B8093C5049093C6042A
:102B3000A093C704B093C80401301105F1F580914A
:102B4000D3049091D404A091D504B091D60480937D
:102B5000A8019093A901A093AA01B093AB01409161
:102B600065015091660160916701709168018091E3
:102B70006B0190916C01A0916D01B0916E01841B6D
:102B8000950BA60BB70B80936B0190936C01A093F0
:102B90006D01B0936E010BC00130110571F4C130AD
:102BA000D10509F483CFCF3FEFEFDE0741F26BE6AB
:102BB00071E08AE190E00E941E118091D80490910A
:102BC000D904029709F06FC0C130D10529F5809171
:102BD000D3049091D404A091D504B091D6048093ED
:102BE000A8019093A901A093AA01B093AB01809191
:102BF000650190916601A0916701B09168014091D3
:102C0000AC015091AD016091AE017091AF01840FA4
:102C1000951FA61FB71F39C0CF3FFFEFDF07E9F5AC
:102C20008091AC019091AD01A091AE01B091AF0146
:102C30004091A3015091A4016091A5017091A6015A
:102C4000480F591F6A1F7B1F4038534C694C714015
:102C500024F14091D3045091D4046091D504709133
:102C6000D6044093A8015093A9016093AA017093E0
:102C7000AB014091650150916601609167017091CF
:102C80006801841B950BA60BB70B8093AC01909346
:102C9000AD01A093AE01B093AF016CEA71E08FE09B
:102CA00090E00E941E118091D8049091D90403975E
:102CB00009F065C0C130D10529F58091D304909108
:102CC000D404A091D504B091D6048093A801909328
:102CD000A901A093AA01B093AB01809165019091E5
:102CE0006601A0916701B09168014091A3015091E4
:102CF000A4016091A5017091A601840F951FA61FE4
:102D0000B71F2FC0CF3F8FEFD80799F58091A30150
:102D10009091A401A091A501B091A601813AE6E8A5
:102D20009E07E1E0AE07B10524F14091D304509134
:102D3000D4046091D5047091D6044093A8015093B7
:102D4000A9016093AA017093AB0140916501509174
:102D500066016091670170916801841B950BA60B59
:102D6000B70B8093A3019093A401A093A501B09306
:102D7000A60163EA71E085E190E00E941E11809156
:102D8000D8049091D904049709F03FC08091D304EE
:102D90009091D404A091D504B091D6048093A80159
:102DA0009093A901A093AA01B093AB01C130D105C2
:102DB00091F48093A8019093A901A093AA01B093E4
:102DC000AB0166E572E08DE696E00E94990E81E027
:102DD0008093A70114C0CF3FFFEFDF0781F48093FA
:102DE000A8019093A901A093AA01B093AB0162E559
:102DF00072E08DE696E00E94990E1092A70167EAB4
:102E000071E08DE090E00E9478118091D80490915B
:102E1000D904059709F03FC08091D3049091D40460
:102E2000A091D504B091D6048093A8019093A901F4
:102E3000A093AA01B093AB01C130D10591F4809366
:102E4000A8019093A901A093AA01B093AB0166E5F4
:102E500072E083E796E00E94990E81E08093B001D2
:102E600014C0CF3F2FEFD20781F48093A801909335
:102E7000A901A093AA01B093AB0162E572E083E7D8
:102E800096E00E94990E1092B00160EB71E080E034
:102E900090E00E9478118091D8049091D90406970F
:102EA00009F072C0C130D10541F58091D3049091F1
:102EB000D404A091D504B091D6048093A801909336
:102EC000A901A093AA01B093AB016BE971E088E27C
:102ED00090E00E94F8104091650150916601609168
:102EE000670170916801FC0180819181A281B381A9
:102EF000840F951FA61FB71F30C0CF3FFFEFDF071E
:102F0000E9F58091D3049091D404A091D504B091B7
:102F1000D6048093A8019093A901A093AA01B0932D
:102F2000AB016BE971E088E290E00E94F8104091FB
:102F30006501509166016091670170916801FC0123
:102F400080819181A281B381841B950BA60BB70B65
:102F5000181619061A061B064CF480939B019093D1
:102F60009C01A0939D01B0939E0108C010929B010B
:102F700010929C0110929D0110929E016BE971E0EC
:102F800088E290E00E941E118091D8049091D904AB
:102F9000079709F05EC0C130D10529F58091D304AF
:102FA0009091D404A091D504B091D6048093A80147
:102FB0009093A901A093AA01B093AB018091650100
:102FC00090916601A0916701B09168014091CF0492
:102FD0005091D0046091D1047091D204840F951F58
:102FE000A61FB71F28C0CF3FFFEFDF0761F5809115
:102FF000D3049091D404A091D504B091D6048093C9
:10300000A8019093A901A093AA01B093AB014091AC
:10301000650150916601609167017091680180912E
:10302000CF049091D004A091D104B091D204841B1C
:10303000950BA60BB70B8093CF049093D004A0936D
:10304000D104B093D2046FEC74E084E290E00E946B
:103050001E118091D8049091D904079779F5CF3F3C
:103060002FEFD20799F48091D3049091D404A091CA
:10307000D504B091D6048093A8019093A901A093A0
:10308000AA01B093AB0162E572E014C02197B1F4DC
:103090008091D3049091D404A091D504B091D6042A
:1030A0008093A8019093A901A093AA01B093AB01CA
:1030B00066E572E087E696E00E94990E8091D8045A
:1030C0009091D904099781F4DF91CF911F910F91CD
:1030D000FF90BF90AF909F908F900C945212013050
:1030E000110509F06ACD63CDDF91CF911F910F914A
:1030F000FF90BF90AF909F908F9008958091B904FA
:103100009091BA04892BD9F460E271E08AEA90E0E8
:103110000E94F810FC0180819181A281B38180938B
:10312000A8019093A901A093AA01B093AB011092BA
:10313000C5041092C6041092C7041092C80480916E
:10314000B9049091BA040197D9F46CE171E08FEA67
:1031500090E00E94F810FC0180819181A281B381EE
:103160008093A8019093A901A093AA01B093AB0109
:103170001092C5041092C6041092C7041092C8049D
:103180008091B9049091BA040297D9F468E171E092
:1031900084EB90E00E94F810FC0180819181A28173
:1031A000B3818093A8019093A901A093AA01B09341
:1031B000AB011092C5041092C6041092C70410927D
:1031C000C8048091B9049091BA040397D9F464E1DA
:1031D00071E089EB90E00E94F810FC018081918100
:1031E000A281B3818093A8019093A901A093AA0121
:1031F000B093AB011092C5041092C6041092C7049C
:103200001092C8048091B9049091BA040497D9F43B
:1032100060E171E08EEB90E00E94F810FC0180818B
:103220009181A281B3818093A8019093A901A09379
:10323000AA01B093AB011092C5041092C60410927B
:10324000C7041092C8048091B9049091BA040597FC
:10325000D9F46CE071E083EC90E00E94F810FC017E
:1032600080819181A281B3818093A8019093A9016B
:10327000A093AA01B093AB011092C5041092C604AA
:103280001092C7041092C8048091B9049091BA04B6
:103290000697D9F468E071E088EC90E00E94F8109D
:1032A000FC0180819181A281B3818093A8019093D8
:1032B000A901A093AA01B093AB011092C50410928A
:1032C000C6041092C7041092C8048091B90490916A
:1032D000BA040797D9F464E071E08DEC90E00E94A5
:1032E000F810FC0180819181A281B3818093A801B3
:1032F0009093A901A093AA01B093AB011092C504C9
:103300001092C6041092C7041092C8048091B904A8
:103310009091BA040897D9F460E071E082ED90E0F2
:103320000E94F810FC0180819181A281B381809379
:10333000A8019093A901A093AA01B093AB011092A8
:10334000C5041092C6041092C7041092C80480915C
:10335000B9049091BA040997D9F461EB71E087ED53
:1033600090E00E94F810FC0180819181A281B381DC
:103370008093A8019093A901A093AA01B093AB01F7
:103380001092C5041092C6041092C7041092C8048B
:1033900008958091BB049091BC0461E0019709F409
:1033A00050C080E00E94DB1B809165019091660116
:1033B000A0916701B091680184369105A105B1051E
:1033C00089F188F48A309105A105B10529F182338C
:1033D0009105A105B10519F10197A105B105C1F547
:1033E00087E794E033C0883E23E09207A105B1054A
:1033F000F9F030F4843F9140A105B105B1F0089592
:10340000803127E29207A105B105A9F0803A9648DC
:10341000A140B10599F008958CE794E017C081E8C8
:1034200094E014C086E894E011C08BE894E00EC0EC
:1034300080E994E00BC085E994E008C08AE994E053
:1034400005C080E00E94DB1B8FE994E00C94D91B3F
:10345000089561E084E00E94DB1B6091A3017091FC
:10346000A4018091A5019091A6016093C10470937D
:10347000C2048093C3049093C40420E432E44FE078
:1034800050E00E94A5332093BD043093BE044093C6
:10349000BF045093C0040E949A1180E20C94ED1B6B
:1034A00060E083E00E94DB1B8091A8019091A9015C
:1034B000A091AA01B091AB018093C1049093C20482
:1034C000A093C304B093C4046091A8017091A901B2
:1034D0008091AA019091AB0120E432E44FE050E0EA
:1034E0000E9483332093BD043093BE044093BF04F5
:1034F0005093C00480E20E94ED1B0E949A1160E08C
:103500008FE00E94DB1B63EA76E08AEE96E00C9483
:10351000CA0E1F920F920FB60F921124CF92DF9214
:10352000EF92FF920F931F932F933F934F935F93CD
:103530006F937F938F939F93AF93BF93CF93DF93BB
:10354000EF93FF938091AB060E94A30BEC01809157
:10355000AA060E94A30BE091A906EF70CC0FDD1F15
:103560008C2B94E0E99FF0011124E554FE4FE80F05
:10357000F11DC081C093A906C07359F10E94621E5B
:103580000091B0041091B1042091B2043091B304C1
:103590006B017C01C01AD10AE20AF30AC092B4049A
:1035A000D092B504E092B604F092B7046093B004F0
:1035B0007093B1048093B2049093B304C03119F4B2
:1035C00081E090E004C0C03221F48FEF9FEF0E94B1
:1035D0004B14FF91EF91DF91CF91BF91AF919F91EC
:1035E0008F917F916F915F914F913F912F911F919B
:1035F0000F91FF90EF90DF90CF900F900FBE0F9044
:103600001F901895FF920F931F93CF93DF93EC01B8
:10361000F62E08811981C8010E94E031F81621F0C8
:103620006F2DC8010E94E831CE01DF91CF911F912B
:103630000F91FF900895009769F0FC010190002020
:10364000E9F73197AF01481B590BBC018AEE96E0B0
:103650000C942E0C80E090E0089540E0682F8AEEF4
:1036600096E00C945D0FCF93DF93823028F0909119
:10367000F90698609093F9068093FD061092FE0675
:1036800080E48093FF0680E18093000780E58093CB
:10369000010761E08091EE060E94D51D8091EF0642
:1036A0008F3F19F061E00E94D51D61E08091F00626
:1036B0000E94D51DCAEED6E09E012A5E364080915A
:1036C000F90684FD03C084E090E002C088E090E049
:1036D0002196281739072CF461E08E810E94D51DB0
:1036E000EBCF8BE39DE00197F1F760E08091EE0670
:1036F0000E94CC0B60E08091F0060E94CC0B809180
:10370000EF068F3F19F060E00E94CC0B8091F90624
:1037100084FD20C063E08AEE96E00E94300FCBE487
:10372000D6E4CE010197F1F763E08AEE96E00E94BD
:10373000300F2197F1F763E08AEE96E00E94300F98
:1037400083E592E00197F1F762E08AEE96E00E944D
:10375000300F15C080620E942D1B8BE496E4019708
:10376000F1F78091F90680620E942D1B83E592E0BB
:103770000197F1F78091F90680620E942D1B8091DC
:10378000F90680620E942D1B84E08093FA068CE08B
:103790000E942D1B81E00E942D1B8BE39FE101976E
:1037A000F1F782E08093FB0686E0DF91CF910C94E5
:1037B0002D1B0C941B1B643008F063E09091FD06F8
:1037C000691710F06FEF690FE62FF0E0E651F94F3F
:1037D0009489890F80680C942D1B41E0682F8AEE34
:1037E00096E00E945D0F81E090E008958F929F9295
:1037F000AF92BF920F931F93CF93DF93CDB7DEB7F6
:10380000A1970FB6F894DEBF0FBECDBF19A242300C
:1038100008F44AE08E010F5D1F4F842E912CA12CDD
:10382000B12CA50194010E948333E62FB901CA018E
:1038300001501109EA3014F4E05D01C0E95CD801DF
:10384000EC93232B242B252B61F7C8010E941B1B13
:10385000A1960FB6F894DEBF0FBECDBFDF91CF911A
:103860001F910F91BF90AF909F908F9008958F926E
:103870009F92AF92BF92CF92DF92EF92FF920F93FF
:103880001F93CF93DF936B017C01142F9B01AC013D
:103890000E945A33882319F084EA94E027C0460135
:1038A0005701E894B7F82FEF3FEF4FE75FE7C50107
:1038B000B4010E945A3381110DC02FEF3FEF4FE743
:1038C0005FE7C501B4010E94BC3018161CF488EAF9
:1038D00094E00CC02FEF3FEF4FE75FE4C701B60164
:1038E0000E945533181684F48CEA94E0DF91CF914E
:1038F0001F910F91FF90EF90DF90CF90BF90AF900E
:103900009F908F900C941B1B2FEF3FEF4FE75FECC6
:10391000C701B6010E94BC3087FDE6CF20E030E051
:10392000A901C701B6010E94BC3087FF09C08DE222
:103930000E94ED1BEC01F7FAF094F7F8F09402C046
:10394000C0E0D0E000E060E070E080E09FE31017AE
:1039500041F020E030E040E251E40E94B4320F5FD9
:10396000F6CFA70196010E9448326B017C010E94AC
:1039700026334B015C014AE00E94F61BC80FD91F99
:103980001123A9F1C501B4010E94C1309B01AC0112
:10399000C701B6010E9447326B017C018EE20E9492
:1039A000ED1BC80FD91F20E030E040E251E4C70111
:1039B000B6010E9422314B015C010E9426336B014B
:1039C000E12CF12C4AE0C701B6010E94F61BC80F9A
:1039D000D91FC701B6010E94C1309B01AC01C501CE
:1039E000B4010E9447326B017C011150E1F6CE0117
:1039F000DF91CF911F910F91FF90EF90DF90CF90CB
:103A0000BF90AF909F908F900895282F3091BD0563
:103A1000313208F04AC0809199058111FCCF909114
:103A2000BC0542E040939905209398052FEF209321
:103A300097051092960530939505ECE9F5E0A5E71A
:103A4000B5E020E0321721F041914D932F5FFACF7E
:103A50001092740520917405990F922B9093740520
:103A600090917305913061F41092730590917405F3
:103A70009093BB009091BC0093FDF8CF95EC01C0F2
:103A800095EE9093BC00909199059230E1F390915E
:103A900097059F3F79F080919705803241F08091A2
:103AA0009705803331F084E005C081E003C082E0F7
:103AB00001C083E010929B051092BD0510929A05FB
:103AC00008950F931F93CF93DF938B0191E0909311
:103AD0009A0590E69093BC0510929B051092BD0547
:103AE000682F8BE596E00E94C70DE801085F1F4F25
:103AF00069918BE596E00E94C70DC017D107C1F709
:103B000081E0DF91CF911F910F910C94051D3FB77C
:103B1000F8948091070790910807A0910907B09148
:103B20000A0726B5A89B05C02F3F19F00196A11DD5
:103B3000B11D3FBFBA2FA92F982F8827820F911D43
:103B4000A11DB11DBC01CD0142E0660F771F881F8A
:103B5000991F4A95D1F70895833081F028F4813078
:103B600099F08230A1F008958730A9F08830B9F03B
:103B70008430D1F4809180008F7D03C080918000DB
:103B80008F7780938000089584B58F7702C084B5C5
:103B90008F7D84BD08958091B0008F7703C08091A0
:103BA000B0008F7D8093B0000895CF93DF9390E0B5
:103BB000FC01E055FF4F2491FC01E456FF4F849136
:103BC000882361F190E0880F991FFC01E852FF4FB4
:103BD000C591D491FC01E857FF4FA591B4916111B3
:103BE00009C09FB7F8948881209582238883EC913F
:103BF0002E230BC0623061F49FB7F8948881322F76
:103C0000309583238883EC912E2B2C939FBF06C085
:103C10008FB7F894E8812E2B28838FBFDF91CF9147
:103C200008958E3008F08E508770806480937C00F9
:103C300080917A00806480937A0080917A0086FD7A
:103C4000FCCF809178002091790090E0922B08952C
:103C50008F929F92AF92BF92CF92DF92EF92FF929C
:103C60006B017C010E94871D4B015C01C114D104D2
:103C7000E104F104F1F00E94871DDC01CB018819F9
:103C80009909AA09BB09883E9340A105B10570F3C3
:103C900021E0C21AD108E108F10888EE880E83E01D
:103CA000981EA11CB11CC114D104E104F10419F740
:103CB000DDCFFF90EF90DF90CF90BF90AF909F90BF
:103CC0008F9008952FB7F8946091030770910407BF
:103CD00080910507909106072FBF08951F920F92BC
:103CE0000FB60F9211242F933F938F939F93AF930F
:103CF000BF938091030790910407A0910507B091AD
:103D000006073091020723E0230F2D3720F4019698
:103D1000A11DB11D05C026E8230F0296A11DB11DEE
:103D2000209302078093030790930407A09305074D
:103D3000B09306078091070790910807A0910907A3
:103D4000B0910A070196A11DB11D809307079093BA
:103D50000807A0930907B0930A07BF91AF919F91FD
:103D60008F913F912F910F900FBE0F901F9018953C
:103D7000CF93DF93CDB7DEB7AB970FB6F894DEBF26
:103D80000FBECDBF789484B5826084BD84B5816058
:103D900084BD85B5826085BD85B5816085BD809116
:103DA0006E00816080936E0010928100809181008E
:103DB0008260809381008091810081608093810086
:103DC000809180008160809380008091B100846048
:103DD0008093B1008091B00081608093B0008091A9
:103DE0007A00846080937A0080917A008260809368
:103DF0007A0080917A00816080937A0080917A00C5
:103E0000806880937A001092C100E091CE05F09115
:103E1000CF0582E08083E091CA05F091CB05108246
:103E2000E091CC05F091CD058FEC80831092D60502
:103E3000E091D205F091D30586E08083E091D00532
:103E4000F091D105808180618083E091D005F0916F
:103E5000D105808188608083E091D005F091D10503
:103E6000808180688083E091D005F091D1058081C8
:103E70008F7D808382E00E94331B81E00E942D1B96
:103E80008BE39FE10197F1F70E94FB0B61E08AE071
:103E90000E94D51D61E08BE00E94D51D61E08CE0A1
:103EA0000E94D51D61E08DE00E94D51D60E08FE08D
:103EB0000E94D51D61E080E10E94D51D61E081E195
:103EC0000E94D51D68E571E081E00E94860B60E5E7
:103ED00071E082E00E94860B68E471E083E00E945A
:103EE000860B60E471E084E00E94860B68E371E079
:103EF00085E00E94860B60E371E086E00E94860BFD
:103F000068E271E087E00E94860B6EED74E089E064
:103F100090E00E949011DC018C918A3809F0CAC3AC
:103F20008EE00E94111E853F91403CF08EE00E9481
:103F3000111E8A3892400CF4BDC36AED74E08FE024
:103F400090E00E94F810FC0180819181A281B381F0
:103F50008093AC019093AD01A093AE01B093AF01FB
:103F600060EB71E080E090E00E949011DC018C91A8
:103F70008093B00165EF74E085E190E00E94F81055
:103F8000FC0180819181A281B3818093A3019093F0
:103F9000A401A093A501B093A60167EA71E08DE0AA
:103FA00090E00E949011DC018C918093A7016BE658
:103FB00071E08AE190E00E94F810FC01808191811B
:103FC000A281B38180936B0190936C01A0936D01EA
:103FD000B0936E0160E671E08FE190E00E94F8100E
:103FE000FC0180819181A281B3818093A80190938B
:103FF000A901A093AA01B093AB016FEC74E084E235
:1040000090E00E94F810FC0180819181A281B3812F
:1040100080939F019093A001A093A101B093A2016E
:104020006BE971E088E290E00E94F810FC01808169
:104030009181A281B38180939B0190939C01A09375
:104040009D01B0939E0169E671E087E390E00E94D4
:10405000E410DC018D919C9190936A018093690139
:1040600080916B0190916C01A0916D01B0916E01F6
:104070008093E0069093E106A093E206B093E306F6
:104080000E94FB0B62E987EB0E94C30560E880E1B8
:104090000E94C30560E881E10E94C30560E882E1F7
:1040A0000E94C3056CE080E10E94C3056CE081E1E1
:1040B0000E94C3056CE082E10E94C30560E281EBCF
:1040C0000E94C30560E881EB0E94C30500E010E098
:1040D00020E03EE249E556E761E170E080E090E0F3
:1040E0000E94240461E081E090E00E94230B80E0C4
:1040F00090E00E947A0B81E090E00E947A0B82E0CF
:1041000090E00E947A0B67E072E083EA96E00E94FA
:10411000990E62E08EE00E94D51D80916800846057
:104120008093680080916D008C6080936D0078941E
:104130000E94621E6093B0047093B1048093B20435
:104140009093B30488EE93E0A0E0B0E08093B404D1
:104150009093B504A093B604B093B7040E94501A8C
:10416000FF24F39464E671E088E090E00E949011EF
:10417000FC0180818093640181110CC061E972E0CF
:104180008DE996E00E94990EF092F30461E080E1DF
:104190000E94CC0B80916401813061F469E072E08F
:1041A0008DE996E00E94990E1092F30460E080E1A0
:1041B0000E94CC0B60E671E08FE190E00E94F81065
:1041C000FC0180819181A281B381809360019093F1
:1041D0006101A0936201B093630160E671E08FE139
:1041E00090E00E94F810DC014D915D916D917C9101
:1041F0008091A8019091A901A091AA01B091AB0171
:10420000481759076A077B0731F068EA71E08FE1C8
:1042100090E00E941E118091BB049091BC04019714
:1042200009F097C08091B4049091B504A091B604B0
:10423000B091B70485369105A105B105C0F02AE01B
:1042400030E040E050E020936501309366014093F8
:104250006701509368018EE690E0A0E0B0E08093A3
:10426000B4049093B504A093B604B093B7048091BE
:10427000B4049091B504A091B604B091B7048997A5
:10428000A109B109CC97A105B105C0F422E330E042
:1042900040E050E020936501309366014093670150
:1042A0005093680186E490E0A0E0B0E08093B4040D
:1042B0009093B504A093B604B093B7048091B4046E
:1042C0009091B504A091B604B091B7044F97A1099D
:1042D000B1090A97A105B105C0F424E630E040E039
:1042E00050E020936501309366014093670150933D
:1042F000680183E290E0A0E0B0E08093B404909382
:10430000B504A093B604B093B7048091B40490911F
:10431000B504A091B604B091B7044F97A105B105BB
:10432000C0F428EE33E040E050E020936501309384
:10433000660140936701509368018FE090E0A0E030
:10434000B0E08093B4049093B504A093B604B09306
:10435000B7048091D8049091D904892B11F40E945C
:10436000501A8EE00E94111E8EE00E94111E5C0108
:104370009093E2048093E1046AE070E080E090E0D2
:104380000E94281E8EE00E94111E8EE00E94111EC7
:10439000092E000CAA0BBB0BA5010B2C000C660B05
:1043A000770B2C013D01E3E04E1A510861087108BA
:1043B000441555056605770564F00396A11DB11DEA
:1043C00084179507A607B70724F0B092E804A092D7
:1043D000E704A090E704B090E804F5E8AF16F3E036
:1043E000BF066CF01092E0048091DF04811145C19A
:1043F00060E081E10E94CC0B109205053EC128E4EB
:10440000A216B10464F48091E004811108C061E057
:1044100081E10E94CC0BF0920505F092E004C50109
:10442000895491098D34910520F58091E004811122
:1044300020C08091DF0481110AC061E081E10E9407
:10444000CC0BF092DF04F0920505F092E00480912D
:10445000E004811112C11091DF04113009F00DC187
:1044600060E081E10E94CC0B1092DF041092050500
:104470008CC0C501875991098034910500F5809160
:10448000E00481111CC08091D704811108C0F09212
:10449000D704F092E0041092E6041092E5048091B3
:1044A000E00481110CC08091D704813041F4109256
:1044B000D7048093E0041092E6041092E504C5014D
:1044C000885D9109C697B8F48091E004811113C00A
:1044D0008091B9049091BA0401968830910514F046
:1044E00088E090E09093BA048093B904F092E004DD
:1044F0000E947E18C2C0C5018F509140C19788F4B8
:104500008091E00481110DC08091B9049091BA04AA
:1045100001971816190634F31092BA041092B904D0
:10452000E5CFC501815491408C9790F58091E004CE
:1045300081112EC08091F304811110C061E080E1EF
:104540000E94CC0B1092640164E671E088E090E078
:104550000E947811F092F304F092E0048091E0045C
:1045600081118BC01091F304113009F086C060E016
:1045700080E10E94CC0B1093640164E671E088E056
:1045800090E00E9478111092F3041093E00475C03B
:10459000C5018E5691408297D0F48091E00481113C
:1045A00016C08091F404811104C0F092F404F092DA
:1045B000E0048091E004811160C08091F4048130B6
:1045C00009F05BC01092F4048093E00456C0C5016A
:1045D000815991408297D8F48091E004811117C0ED
:1045E0008091690190916A0101968830910514F0DB
:1045F00088E090E090936A0180936901F092E00472
:1046000069E671E087E390E00E94511136C0C50170
:104610008F5A91408336910588F48091E00481118E
:104620000DC08091690190916A01019718161906D1
:104630000CF310926A0110926901E0CF33E1A31AE2
:1046400032E0B30A47E7A416B104B8F48091E0045D
:10465000811113C08091D8049091D9040196909350
:10466000D9048093D804F092B804099724F01092EA
:10467000D9041092D804F092E0048091A80190919E
:10468000A901A091AA01B091AB018032914AA74043
:10469000B10508F40BC18091A8019091A901A091E6
:1046A000AA01B091AB018038994BAA42B10508F438
:1046B00026C1FCC060EB71E080E090E00E947811C0
:1046C0008AE890E09A838983BE016F5F7F4F89E01B
:1046D00090E00E94511167EA71E08DE090E00E9445
:1046E00078116CEA71E08FE090E00E941E1163EA9D
:1046F00071E085E190E00E941E116BE671E08AE1B5
:1047000090E00E941E1168EA71E08FE190E00E9443
:104710001E116FE971E084E290E00E941E116BE9C6
:1047200071E088E290E00E941E1169E671E087E383
:1047300090E00E94511166E271E084E690E00E94F0
:10474000511164E271E087E690E00E9451116FE63A
:1047500071E08AE690E00E94511161E771E08DE618
:1047600090E00E94511163E771E080E790E00E94C1
:10477000511165E771E083E790E00E94511167E70E
:1047800071E086E790E00E94511169E771E089E7E6
:1047900090E00E9451116BE771E08CE790E00E947D
:1047A00051116DE771E08FE790E00E9451116FE7C2
:1047B00071E082E890E00E94511161E871E085E8C3
:1047C00090E00E94511163E871E088E890E00E9457
:1047D000511165E871E08BE890E00E94511167E8A3
:1047E00071E08EE890E00E94511169E871E081E982
:1047F00090E00E9451116BE871E084E990E00E9422
:1048000051116DE871E087E990E00E9451116FE865
:1048100071E08AE990E00E94511161E971E08DE94F
:1048200090E00E94511163E971E080EA90E00E94FB
:10483000511165E971E083EA90E00E94511160E254
:1048400071E08AEA90E00E941E116CE171E08FEA4B
:1048500090E00E941E1168E171E084EB90E00E94FC
:104860001E1164E171E089EB90E00E941E1160E18D
:1048700071E08EEB90E00E941E116CE071E083EC21
:1048800090E00E941E1168E071E088EC90E00E94C8
:104890001E1164E071E08DEC90E00E941E1160E05A
:1048A00071E082ED90E00E941E1147CB8091A8013B
:1048B0009091A901A091AA01B091AB018038994BC8
:1048C000AA42B10548F18091A8019091A901A09157
:1048D000AA01B091AB0180349B44AC44B105E0F433
:1048E0002A9A2B982C982D9881E090E09093BA0406
:1048F0008093B90468EA71E08FEA90E0DDC02A98FD
:104900002B982C982D981092BA041092B90468EA4A
:1049100071E08AEA90E0D0C08091A8019091A9014D
:10492000A091AA01B091AB0180349B44AC44B10585
:10493000E0F08091A8019091A901A091AA01B09105
:10494000AB0181159241AA47B10578F42A982B9AB8
:104950002C982D9882E090E09093BA048093B9044B
:1049600068EA71E084EB90E0A7C08091A801909183
:10497000A901A091AA01B091AB0181159241AA476A
:10498000B105E0F08091A8019091A901A091AA0140
:10499000B091AB0181159B41A74BB10578F42A9AE0
:1049A0002B9A2C982D9883E090E09093BA048093F2
:1049B000B90468EA71E089EB90E07EC08091A801BB
:1049C0009091A901A091AA01B091AB0181159B41E1
:1049D000A74BB105E0F08091A8019091A901A091A9
:1049E000AA01B091AB0181159442A44FB10578F4AE
:1049F0002A982B982C9A2D9884E090E09093BA04F2
:104A00008093B90468EA71E08EEB90E055C0809124
:104A1000A8019091A901A091AA01B091AB018115C3
:104A20009442A44FB105E0F08091A8019091A901B2
:104A3000A091AA01B091AB01803C9A4EA142B14035
:104A400078F42A9A2B982C9A2D9885E090E09093F0
:104A5000BA048093B90468EA71E083EC90E02CC05A
:104A60008091A8019091A901A091AA01B091AB01F8
:104A7000803C9A4EA142B14010F40C946D2E80916E
:104A8000A8019091A901A091AA01B091AB01803831
:104A9000914BAF44B14010F00C946D2E2A982B9A94
:104AA0002C9A2D9886E090E09093BA048093B904F4
:104AB00068EA71E088EC90E00E941E118091690123
:104AC00090916A01009739F421E030E03093BC0402
:104AD0002093BB0444C08130910589F421E030E08B
:104AE00040E050E0209365013093660140936701F8
:104AF000509368011092BC041092BB0430C0823005
:104B0000910589F42AE030E040E050E0209365010F
:104B10003093660140936701509368011092BC0482
:104B20001092BB0424C08330910589F422E330E065
:104B300040E050E0209365013093660140936701A7
:104B4000509368011092BC041092BB0418C08430CA
:104B5000910529F484E690E0A0E0B0E026C085301D
:104B6000910529F424EF31E040E050E00FC0863099
:104B7000910529F488EE93E0A0E0B0E016C08730FC
:104B8000910569F420E137E240E050E020936501AF
:104B90003093660140936701509368010EC00897F7
:104BA00081F480EA96E8A1E0B0E0809365019093FB
:104BB0006601A0936701B09368011092BC04109243
:104BC000BB048091D8049091D904181619060CF0F2
:104BD00091C1019701F560E080E00E94DB1B8DE050
:104BE00092E00E94D91B0E94C91961E084E00E94F2
:104BF000DB1B8CE693E00E94D91B60916B017091E6
:104C00006C0180916D0190916E010E94500B8BE9B7
:104C100093E00E94D91B8091D8049091D904029707
:104C200089F560E080E00E94DB1B8FE192E00E944A
:104C3000D91B0E94C91961E084E00E94DB1B6091CE
:104C4000AC017091AD018091AE019091AF01609384
:104C5000C1047093C2048093C3049093C40420E4FD
:104C600032E44FE050E00E94A5332093BD0430931E
:104C7000BE044093BF045093C0040E949A1180E286
:104C80000E94ED1B8091D8049091D904039761F4A0
:104C90000E94291A60E080E00E94DB1B80E392E022
:104CA0000E94D91B0E94C9198091D8049091D904FF
:104CB000049759F50E94291A60E080E00E94DB1BEE
:104CC00081E492E00E94D91B8091A701811106C066
:104CD00062E572E08DE696E00E94990E8091A70150
:104CE000813031F466E572E08DE696E00E94990E1F
:104CF00061E080E00E94DB1B6DE676E08AEE96E0E4
:104D00000E94CA0E80E20E94ED1B8091D80490910F
:104D1000D904059709F04DC060E080E00E94DB1BDC
:104D20008AE592E00E94D91B8091B001811106C0F2
:104D300062E572E083E796E00E94990E8091B001EF
:104D4000813031F466E572E083E796E00E94990EC7
:104D500061E080E00E94DB1B63E776E08AEE96E08C
:104D60000E94CA0E6091AC017091AD018091AE01BC
:104D70009091AF016093C1047093C2048093C30407
:104D80009093C40420E432E44FE050E00E94A53345
:104D90002093BD043093BE044093BF045093C004DD
:104DA0000E949A118DE693E00E94D91B80E20E9436
:104DB000ED1B8091D8049091D904069719F560E015
:104DC00080E00E94DB1B8BE692E00E94D91B0E94D0
:104DD000C91961E084E00E94DB1B8CE693E00E942D
:104DE000D91B60919B0170919C0180919D019091D4
:104DF0009E010E94500B8CE792E00E94D91B80E23A
:104E00000E94ED1B8091D8049091D904079701F579
:104E100060E080E00E94DB1B84E892E00E94D91BE6
:104E20000E94C91961E084E00E94DB1B8CE693E0DC
:104E30000E94D91B6091CF047091D0048091D1045D
:104E40009091D2040E94500B8CE792E00E94D91BF3
:104E50008091D8049091D9040897F1F460E080E043
:104E60000E94DB1B85E992E00E94D91B8CE693E04F
:104E70000E94D91B61E080E00E94DB1B8FE893E079
:104E80000E94D91B67E676E08AEE96E00E94CA0E81
:104E900083E893E00E94D91B8091D8049091D904B3
:104EA000099741F580916B0690916C06892B11F161
:104EB000A0906706B090680662E572E0C5010E94A6
:104EC0005B37892B21F41092D9041092D80466E53F
:104ED00072E0C5010E945B37892B11F40E945212C7
:104EE0008091D8049091D9040A9724F01092D904A3
:104EF0001092D80480910505813009F0D0C08091CE
:104F0000D8049091D904892B09F0C9C0A090E3047A
:104F1000B090E40485010F5F1F4F1093E4040093E9
:104F2000E30484E10E94111EBC01990F880B990BC8
:104F30000E94C3304B015C0185E10E94111EBC013F
:104F4000990F880B990B0E94C3302B013C019B01E8
:104F5000AC01C501B4010E94553387FD07C061E073
:104F600080E00E94DB1B85EA92E097C004311105C6
:104F70000CF495C01092E4041092E304A301920192
:104F8000C501B4010E94483268A779A78AA79BA7E8
:104F9000A5019401C301B2010E9447329B01AC01FB
:104FA00068A579A58AA59BA50E94B4324B015C0136
:104FB00020E030E0A9010E945533181624F0B7FA1A
:104FC000B094B7F8B09420E030E040EA50E4C30178
:104FD000B2010E94223120E030EC4FE754E40E94FD
:104FE000B4322CE238E540EB5CE30E94B4329B0122
:104FF000AC010E94223120E030E048E452E40E94FB
:10500000B4322B013C0120E030E040E050E4C50127
:10501000B4010E94483268A779A78AA79BA7A50177
:10502000940160E070E080E89FE30E94B4329B014D
:10503000AC0168A579A58AA59BA50E9448329B0171
:10504000AC0160E070E080E890E40E94B432A3011B
:1050500092010E9422312B013C0161E080E00E941C
:10506000DB1B88EB92E00E94D91B42E0C501B40132
:105070000E94371C61E088E00E94DB1B8DEB92E010
:105080000E94D91B61E08BE00E94DB1B40E0C30162
:10509000B2010E94371C81EC92E00E94D91B91E082
:1050A0008091D704813009F090E081E020910505DE
:1050B000211180E0892309F4ABC08091D80490913C
:1050C000D904892B09F0A4C080919701909198018F
:1050D000A0919901B0919A018032E1EA9E07E7E040
:1050E000AE07B105A4F48091A8019091A901A09107
:1050F000AA01B091AB018052914AA740B109B09585
:10510000A095909581959F4FAF4FBF4F15C08130AF
:10511000914EA54FB540C4F04091A8015091A9010E
:105120006091AA017091AB0180E091EEA5EFB5E02E
:10513000841B950BA60BB70B8093C5049093C604F4
:10514000A093C704B093C8048091E7049091E80449
:1051500087599109C197D0F48091E5049091E604B4
:10516000843691059CF401969093E6048093E504BF
:10517000C29761F41092C5041092C6041092C7043D
:105180001092C8041092E6041092E5040E94C91916
:105190008090A8019090A901A090AA01B090AB01C5
:1051A0008091C5049091C604A091C704B091C80431
:1051B000880E991EAA1EBB1E80929701909298019C
:1051C000A0929901B0929A0161E084E00E94DB1BF9
:1051D0008092C1049092C204A092C304B092C4040D
:1051E000C501B40120E432E44FE050E00E94A53351
:1051F0002093BD043093BE044093BF045093C00479
:105200000E949A1180E20E94ED1B80E20E94ED1B39
:1052100091E080910505811190E081E02091D70413
:10522000211180E0892309F421C28091D804909152
:10523000D904892B09F01AC26EE673E085E896E07E
:105240000E94990E0E9430120E94621E0E94621EED
:105250008090CB049090CC04A090CD04B090CE046C
:10526000DC01CB0188199909AA09BB09843691058B
:10527000A105B10508F489C50E94621EDC01CB01BD
:1052800088199909AA09BB0984369105A105B105B8
:1052900070F00E94621EDC01CB0188199909AA09ED
:1052A000BB09883C9105A105B10508F477C50E94AA
:1052B000621EDC01CB0188199909AA09BB09883C47
:1052C0009105A105B10570F00E94621EDC01CB01C1
:1052D00088199909AA09BB098C329140A105B10529
:1052E00008F465C50E94621EDC01CB01881999098A
:1052F000AA09BB098C329140A105B10570F00E944A
:10530000621EDC01CB0188199909AA09BB09803901
:105310009140A105B10508F453C50E94621EDC014D
:10532000CB0188199909AA09BB0980399140A105C7
:10533000B10570F00E94621EDC01CB018819990949
:10534000AA09BB09853F9140A105B10508F441C5F3
:105350000E94621EDC01CB0188199909AA09BB09C8
:10536000853F9140A105B10508F47EC12091F1046B
:105370003091F2048091EF049091F004820F931F1A
:105380002091ED043091EE04820F931F2091EB04E5
:105390003091EC04820F931F2091E9043091EA04CC
:1053A000820F931F65E070E00E946F335B01709382
:1053B000CA046093C90465E971E083EA90E00E9441
:1053C000E410DC018D919C91A816B9061CF086ECC6
:1053D00092E034C165E971E083EA90E00E94E41054
:1053E000FC01808191818A159B051CF483ED92E07C
:1053F00025C163E971E080EA90E00E94E410DC01DD
:105400008D919C918A159B051CF480EE92E016C14B
:1054100061E971E08DE990E00E94E410FC01808177
:1054200091818A159B051CF48DEE92E007C16FE80F
:1054300071E08AE990E00E94E410DC018D919C917A
:105440008A159B051CF48AEF92E0F8C06DE871E0C4
:1054500087E990E00E94E410FC01808191818A1527
:105460009B051CF487E093E0E9C06BE871E084E9F8
:1054700090E00E94E410DC018D919C918A159B05BF
:105480001CF484E193E0DAC069E871E081E990E01E
:105490000E94E410FC01808191818A159B051CF417
:1054A00081E293E0CBC067E871E08EE890E00E9473
:1054B000E410DC018D919C918A159B051CF48EE211
:1054C00093E0BCC065E871E08BE890E00E94E410D6
:1054D000FC01808191818A159B051CF48BE393E08C
:1054E000ADC063E871E088E890E00E94E410DC0160
:1054F0008D919C918A159B051CF488E493E09EC0D5
:1055000061E871E085E890E00E94E410FC01808190
:1055100091818A159B051CF485E593E08FC06FE7A8
:1055200071E082E890E00E94E410DC018D919C9192
:105530008A159B051CF482E693E080C06DE771E05C
:105540008FE790E00E94E410FC01808191818A1530
:105550009B051CF48FE693E071C06BE771E08CE76C
:1055600090E00E94E410DC018D919C918A159B05CE
:105570001CF48CE793E062C069E771E089E790E092
:105580000E94E410FC01808191818A159B051CF426
:1055900089E893E053C067E771E086E790E00E94F6
:1055A000E410DC018D919C918A159B051CF486E921
:1055B00093E044C065E771E083E790E00E94E41067
:1055C000FC01808191818A159B051CF483EA93E09C
:1055D00035C063E771E080E790E00E94E410DC01F1
:1055E0008D919C918A159B051CF480EB93E026C05D
:1055F00061E771E08DE690E00E94E410FC0180819B
:1056000091818A159B051CF48DEB93E017C06FE622
:1056100071E08AE690E00E94E410DC018D919C919B
:105620008A159B051CF48AEC93E008C06FE671E0D4
:1056300087E690E00E94E41087ED93E00E943F0B24
:1056400061E084E00E94DB1B65E876E08AEE96E08C
:105650000E94CA0E0E94621E6093CB047093CC0419
:105660008093CD049093CE040E94C9196FEC74E02E
:1056700084E290E00E94F810FC0180819181A28177
:10568000B38180939F019093A001A093A101B09357
:10569000A20165EF74E085E190E00E94F810FC0142
:1056A00080819181A281B3818093A3019093A40111
:1056B000A093A501B093A6016BE971E088E290E0A8
:1056C0000E94F810FC0180819181A281B3818093B6
:1056D0009B0190939C01A0939D01B0939E0110911A
:1056E0000505113081F48091A8019091A901A09144
:1056F000AA01B091AB018093970190939801A09378
:105700009901B0939A018091A8019091A901A0916B
:10571000AA01B091AB0180389F49A54DB105C0F0F9
:105720008091F404811109C067E072E083EA96E099
:105730000E94990E64EE73E0BDC0813049F468EEBA
:1057400073E083EA96E00E94990E6AEE73E01AC055
:105750008091A8019091A901A091AA01B091AB01FB
:1057600080389F49A54DB10508F015C18091F4041A
:10577000811195C068EE73E083EA96E00E94990E6D
:1057800064EE73E087E996E00E94990E9091D70449
:1057900081E02091D8043091D904232B09F080E0D6
:1057A000913001F5882309F45DC04091A301509127
:1057B000A4016091A5017091A6018091AC01909126
:1057C000AD01A091AE01B091AF01840F951FA61F4E
:1057D000B71F8090970190909801A0909901B09088
:1057E0009A0120C091113EC08823E1F14091A301AC
:1057F0005091A4016091A5017091A6018090A8012B
:105800009090A901A090AA01B090AB018091AC0149
:105810009091AD01A091AE01B091AF01840F951FA1
:10582000A61FB71F88199909AA09BB09809301050A
:1058300090930205A0930305B093040580919B010A
:1058400090919C01A0919D01B0919E01480F591F1C
:105850006A1F7B1F4093A3015093A4016093A5018D
:105860007093A6018091F304813009F094C0113047
:1058700009F091C040910105509102056091030526
:105880007091040580919F019091A001A091A101C8
:10589000B091A201840F951FA61FB71F74C081305D
:1058A00009F079C067E072E083EA96E00E94990E01
:1058B0006AEE73E087E996E00E94990E8091D70422
:1058C0008130E9F44091AC015091AD016091AE019D
:1058D0007091AF018091A3019091A401A091A501C5
:1058E000B091A601840F951FA61FB71F4091970185
:1058F000509198016091990170919A011EC0811197
:1059000028C04091A8015091A9016091AA0170910D
:10591000AB018090AC019090AD01A090AE01B09031
:10592000AF018091A3019091A401A091A501B09134
:10593000A601880D991DAA1DBB1D841B950BA60BE6
:10594000B70B8093010590930205A0930305B093D4
:1059500004058091F3048130F1F41130E1F4809179
:10596000010590910205A0910305B09104054091B5
:105970009F015091A0016091A1017091A201841B2F
:10598000950BA60BB70B8093010590930205A0938E
:105990000305B09304058091B001811105C060E05A
:1059A00081E090E00E94230B8091B001813009F0EA
:1059B00087C061E081E090E00E94230B40910105E7
:1059C0005091020560910305709104058091FD04DA
:1059D0009091FE04A091FF04B0910005481759076B
:1059E0006A077B0799F520919B0630919C06809170
:1059F0009506909196062817390741F580919706EC
:105A0000909198066091910670919206009719F016
:105A100061157105B9F46115710551F0232B09F475
:105A20004FC0DB018C9190E09195819591090CC05C
:105A3000009709F445C0232B09F442C0FC01808182
:105A400090E002C00E945B37892BD1F16091AC01DC
:105A50007091AD018091AE019091AF0124E630E0EC
:105A600040E050E00E94233401E010E00E94D406A0
:105A700081E996E0F6E087399F0791F060919706FB
:105A8000709198066115710539F040919B0650910F
:105A90009C060E94780E04C081E996E00E94660E82
:105AA0008091A8019091A901A091AA01B091AB01A8
:105AB0008093D3049093D404A093D504B093D604D8
:105AC0008091A701811105C060E082E090E00E9412
:105AD000230B8091A7018130A1F561E082E090E085
:105AE0000E94230B6091A3017091A4018091A501F4
:105AF0009091A6018090F9049090FA04A090FB0484
:105B0000B090FC04681579058A059B05D1F024E660
:105B100030E040E050E00E94233402E010E00E94B8
:105B2000D4068091A3019091A401A091A501B09108
:105B3000A6018093F9049093FA04A093FB04B09318
:105B4000FC0440910105509102056091030570919C
:105B500004058091FD049091FE04A091FF04B09192
:105B60000005481759076A077B0709F4A2C080910E
:105B7000D8049091D904892B09F09BC06091A801A9
:105B80007091A9018091AA019091AB011BA21AA268
:105B90001DA21CA21FA21EA22AE0AE014F5F5F4FF2
:105BA0000E947030BE016F5F7F4FCE0182960E94CF
:105BB000990E8091790690917A06009709F012C1AA
:105BC0008AA19BA190937A06809379068CA19DA1CE
:105BD00090937C0680937B068EA19FA190937E0676
:105BE00080937D061BA21AA21DA21CA21FA21EA2A8
:105BF000CE0182960E94B00E80917D0690917E0625
:105C00000B9708F408C16EEE73E0CE0101960E9476
:105C1000B50E40917D0650917E0660917906709197
:105C20007A06CE0101960E94380E811104C0CE0181
:105C300001960E94660E41E050E061EF73E0CE01F4
:105C400001960E94380E882309F424C1BE016F5FBB
:105C50007F4F8EEB95E00E94CA0ECE0101960E9406
:105C6000B00E64E170E080E090E00E94281E609138
:105C7000010570910205809103059091040524E6C9
:105C800030E040E050E00E94323400E010E00E943A
:105C9000D4068091010590910205A0910305B09171
:105CA00004058093FD049093FE04A093FF04B09339
:105CB00000058091D8049091D904892B51F460E0BB
:105CC00080E00E94DB1B6DE976E08AEE96E00E94A0
:105CD000CA0E0E94300D0C94B2208091A8019091C0
:105CE000A901A091AA01B091AB018038914BAF44BA
:105CF000B14068F08091A8019091A901A091AA01FA
:105D0000B091AB01803C9C4FAB49B14070F18091A8
:105D1000A8019091A901A091AA01B091AB01803C8A
:105D20009C4FAB49B14010F40C945E258091A801C2
:105D30009091A901A091AA01B091AB018138934C37
:105D4000A94CB14010F00C945E252A982B982C9801
:105D50002D9A88E090E09093BA048093B90468EAA1
:105D600071E082ED90E00C945C252A9A2B9A2C9A93
:105D70002D9887E090E09093BA048093B90468EA84
:105D800071E08DEC90E00C945C258091C9049091B9
:105D9000CA049093F2048093F1046ECA8091C904FE
:105DA0009091CA049093F0048093EF0480CA80918C
:105DB000C9049091CA049093EE048093ED0492CAB2
:105DC0008091C9049091CA049093EC048093EB04F1
:105DD000A4CA8091C9049091CA049093EA04809364
:105DE000E904B6CA6AA17BA16115710509F44FC027
:105DF00040917B0650917C062EA13FA1421753078C
:105E000008F445C00E9464378EA19FA190937E063E
:105E100080937D06EBCE1BA21AA21DA21CA21FA27C
:105E20001EA24AE0BE016F5F7F4F80E090E00E94BB
:105E30006530BE016F5F7F4FCE0182960E94990E42
:105E400040917D0650917E066091790670917A06A8
:105E5000CE0182960E94380E811104C0CE01829636
:105E60000E94660E6AA17BA16115710539F04EA1F1
:105E70005FA189E796E00E94780E04C089E796E06A
:105E80000E94660ECE0182960E94B00EB5CE0E9490
:105E9000FE3596CECE0101960E94660ED7CE87E6DD
:105EA00096E00E94B00E8DE696E00E94B00E83E769
:105EB00096E00E94B00E89E796E00E94B00E8FE750
:105EC00096E00E94B00E85E896E00E94B00E8BE846
:105ED00096E00E94B00E81E996E00E94B00E87E93C
:105EE00096E00E94B00E8DE996E00E94B00E83EA23
:105EF00096E00C94B00ECF93DF93EEEBF5E01382B7
:105F0000128288EE93E0A0E0B0E084839583A683BC
:105F1000B7832BED31E03183208325EC30E03587EA
:105F2000248724EC30E03787268720EC30E0318B63
:105F3000208B21EC30E0338B228B22EC30E0358B50
:105F4000248B26EC30E0378B268B118E128E138E2D
:105F5000148EEBE5F6E01382128284839583A68388
:105F6000B7838DEE91E091838083EAEEF6E01382B1
:105F700012828FEF91E09183808389E084838FEF99
:105F80008583C8E0C68387E0878386E0808785E0D5
:105F9000818784E082871386148615861686178685
:105FA00081E00E94331BECEAF6E0C0AFC1AF11AA5A
:105FB00012AA13AA118612861386148615861686CF
:105FC0001786108A118A128A138A148A158A168AE9
:105FD000178A108E118E128E138E148E158E168EB9
:105FE000178E10A211A212A213A214A215A216A219
:105FF00017A210A611A612A613A614A615A616A6D9
:1060000017A610AA80E498E7ADE7B1E082AF93AF9E
:10601000A4AFB5AFC9EAD6E083E0898382E08A8382
:1060200060E083E00E94D51D60E08A810E94D51D5A
:1060300061E089810E94CC0B61E08A810E94CC0BD7
:10604000188267E072E083EA96E00E94B50E69E08C
:1060500072E08DE996E00E94B50E64EE73E087E988
:1060600096E00E94B50E6EE673E081E996E00E942C
:10607000B50E6EE673E08BE896E00E94B50E6EE614
:1060800073E085E896E00E94B50E6EE673E08FE758
:1060900096E00E94B50E6EE673E089E796E00E94F6
:1060A000B50E66E572E083E796E00E94B50E66E500
:1060B00072E08DE696E00E94B50E62E572E087E63A
:1060C00096E0DF91CF910C94B50EBB274A3031F4A6
:1060D000992322F4BDE2909581959F4F0C949330C3
:1060E000BB27FA01A62F6217710581059105330BB5
:1060F00030FB66F0AA27660F771F881F991FAA1F1B
:10610000A21710F0A21B63953850A9F7A05DAA331F
:1061100008F0A95DA19336F7B111B1931082CA01BD
:106120000C94AC30BB27FB015527AA27880F991F79
:10613000AA1FA41710F0A41B83955051B9F7A05DB6
:10614000AA3308F0A95DA193009779F7B111B19333
:106150001192CB010C94AC30DC01FC01672F7191E2
:106160007723E1F7329704C07C916D93708362913D
:10617000AE17BF07C8F308950E94FE3008F481E00F
:106180000895E89409C097FB3EF49095809570952A
:1061900061957F4F8F4F9F4F9923A9F0F92F96E973
:1061A000BB279395F695879577956795B795F111E8
:1061B000F8CFFAF4BB0F11F460FF1BC06F5F7F4F85
:1061C0008F4F9F4F16C0882311F096E911C0772397
:1061D00021F09EE8872F762F05C0662371F096E8A0
:1061E000862F70E060E02AF09A95660F771F881F6F
:1061F000DAF7880F9695879597F90895990F000813
:10620000550FAA0BE0E8FEEF16161706E807F90788
:10621000C0F012161306E407F50798F0621B730B23
:10622000840B950B39F40A2661F0232B242B252BA4
:1062300021F408950A2609F4A140A6958FEF811D47
:10624000811D08950E9435310C94A6310E94983129
:1062500038F00E949F3120F0952311F00C948F317B
:106260000C94953111240C94DA310E94B73170F3FB
:10627000959FC1F3950F50E0551F629FF001729FEB
:10628000BB27F00DB11D639FAA27F00DB11DAA1FFA
:10629000649F6627B00DA11D661F829F2227B00D47
:1062A000A11D621F739FB00DA11D621F839FA00DD2
:1062B000611D221F749F3327A00D611D231F849F22
:1062C000600D211D822F762F6A2F11249F57504079
:1062D0009AF0F1F088234AF0EE0FFF1FBB1F661FF4
:1062E000771F881F91505040A9F79E3F510580F0BD
:1062F0000C948F310C94DA315F3FE4F3983ED4F381
:10630000869577956795B795F795E7959F5FC1F760
:10631000FE2B880F911D9695879597F9089597F90B
:106320009F6780E870E060E008959FEF80EC08953B
:1063300000240A9416161706180609060895002464
:106340000A9412161306140605060895092E0394DE
:10635000000C11F4882352F0BB0F40F4BF2B11F452
:1063600060FF04C06F5F7F4F8F4F9F4F089557FDB1
:106370009058440F551F59F05F3F71F04795880FB3
:1063800097FB991F61F09F3F79F08795089512164A
:1063900013061406551FF2CF4695F1DF08C01616F6
:1063A00017061806991FF1CF8695710561050894A7
:1063B0000895E894BB2766277727CB0197F90895BE
:1063C000F999FECF92BD81BDF89A992780B50895BD
:1063D000262FF999FECF1FBA92BD81BD20BD0FB601
:1063E000F894FA9AF99A0FBE019608950E943832ED
:1063F000A59F900DB49F900DA49F800D911D112419
:1064000008952F923F924F925F926F927F928F9258
:106410009F92AF92BF92CF92DF92EF92FF920F9333
:106420001F93CF93DF93CDB7DEB7CA1BDB0B0FB63D
:10643000F894DEBF0FBECDBF09942A8839884888FA
:106440005F846E847D848C849B84AA84B984C88490
:10645000DF80EE80FD800C811B81AA81B981CE0F87
:10646000D11D0FB6F894DEBF0FBECDBFED0108956C
:10647000A29FB001B39FC001A39F700D811D112485
:10648000911DB29F700D811D1124911D08955058CA
:10649000BB27AA270E945F320C94A6310E94983134
:1064A00038F00E949F3120F039F49F3F19F426F410
:1064B0000C9495310EF4E095E7FB0C948F31E92FA5
:1064C0000E94B73158F3BA1762077307840795071C
:1064D00020F079F4A6F50C94D9310EF4E0950B2E4A
:1064E000BA2FA02D0B01B90190010C01CA01A00126
:1064F0001124FF27591B99F0593F50F4503E68F181
:106500001A16F040A22F232F342F4427585FF3CFC1
:10651000469537952795A795F0405395C9F77EF492
:106520001F16BA0B620B730B840BBAF09150A1F0DB
:10653000FF0FBB1F661F771F881FC2F70EC0BA0F61
:10654000621F731F841F48F4879577956795B795E9
:10655000F7959E3F08F0B0CF9395880F08F09927E4
:10656000EE0F9795879508950E94C8320C94A63136
:106570000E949F3158F00E94983140F029F45F3F0B
:1065800029F00C948F3151110C94DA310C9495311F
:106590000E94B73168F39923B1F3552391F3951B0A
:1065A000550BBB27AA2762177307840738F09F5F34
:1065B0005F4F220F331F441FAA1FA9F335D00E2EA1
:1065C0003AF0E0E832D091505040E695001CCAF70E
:1065D0002BD0FE2F29D0660F771F881FBB1F2617D1
:1065E00037074807AB07B0E809F0BB0B802DBF01A8
:1065F000FF2793585F4F3AF09E3F510578F00C9477
:106600008F310C94DA315F3FE4F3983ED4F38695F2
:1066100077956795B795F7959F5FC9F7880F911D97
:106620009695879597F90895E1E0660F771F881F83
:10663000BB1F621773078407BA0720F0621B730B36
:10664000840BBA0BEE1F88F7E09508950E94BF31C6
:1066500088F09F5798F0B92F9927B751B0F0E1F023
:10666000660F771F881F991F1AF0BA95C9F714C0D3
:10667000B13091F00E94D931B1E008950C94D93134
:10668000672F782F8827B85F39F0B93FCCF386950C
:1066900077956795B395D9F73EF490958095709569
:1066A00061957F4F8F4F9F4F08950E94FE3008F4F1
:1066B0008FEF08950E94FE30880B990B0895DB013F
:1066C0008F939F930E94F631BF91AF91A29F800D4F
:1066D000911DA39F900DB29F900D1124089597FBDB
:1066E000072E16F4009407D077FD09D00E9452358A
:1066F00007FC05D03EF4909581959F4F08957095C5
:1067000061957F4F0895A1E21A2EAA1BBB1BFD01C4
:106710000DC0AA1FBB1FEE1FFF1FA217B307E40780
:10672000F50720F0A21BB30BE40BF50B661F771FD8
:10673000881F991F1A9469F76095709580959095B8
:106740009B01AC01BD01CF010895052E97FB1EF4FE
:1067500000940E94BC3357FD07D00E94833307FC8E
:1067600003D04EF40C94BC33509540953095219550
:106770003F4F4F4F5F4F089590958095709561956D
:106780007F4F8F4F9F4F0895EE0FFF1F0590F4919D
:10679000E02D0994DF93CF931F930F939A9DF02DD3
:1067A000219FF00D8B9DF00D8A9DE02DF10D039F33
:1067B000F00D029FE00DF11D4E9DE00DF11D5E9D5F
:1067C000F00D4F9DF00D7F936F93BF92AF925F934B
:1067D0004F93D5010E9438328B01AC01D7010E9442
:1067E0003832EB01E80FF91FD6010E941A342F91BD
:1067F0003F91D6010E943832C60FD71FE81FF91FFC
:10680000AF91BF910E941A342F913F910E9438326C
:10681000C60FD71FE81FF91FD6010E943832E60FB6
:10682000F71F9801BE01CF0111240F911F91CF9145
:10683000DF9108950E943832460F571FC81FD91F95
:1068400008F43196089597FB57FF0C9433349F93C7
:106850008F930E9433346E1B7F0BAF91BF918A0BD5
:106860009B0B0895E894DF93CF93FC01DB010E941A
:1068700038327F936F93E9019A01AC01BF93AF93D4
:106880003F932F93DF010E94383226F46C1B7D0B5F
:10689000820B930B9E01EB01FC010E941A34AF9115
:1068A000BF912F913F910E941A34BE01CF01F9018F
:1068B0002F913F91CF91DF910895689401C0E894A2
:1068C000F92FF12B12F00C949134A0E0B0E0EBE63C
:1068D000F4E30C940732092E059422F40E94ED345F
:1068E000112392F4F0E80F26FFEFE094F094009566
:1068F0001095B094C094D094A194BF0ACF0ADF0A37
:10690000EF0AFF0A0F0B1F0B0E949C3407FC0E942A
:10691000ED34CDB7DEB7ECE00C942332689401C0BF
:10692000E8948F929F92CF93DF930E949C34DF91E3
:10693000CF919F908F90089588249924F401E401C9
:10694000B0E49F93AA279A158B049C04ED05FE05DD
:10695000CF05D007A10798F4AD2FDC2FCF2FFE2F46
:10696000E92D982C892E982F872F762F652F542F5D
:10697000432F322F2227B85031F7BF9127C01B2E4B
:10698000BF91BB27220F331F441F551F661F771F60
:10699000881F991F881C991CEE1FFF1FCC1FDD1F2D
:1069A000AA1FBB1F8A149B04EC05FD05CE05DF055D
:1069B000A007B10748F08A189B08EC09FD09CE0929
:1069C000DF09A00BB10B21601A94E1F62EF49401BB
:1069D000AF01BE01CD01000C0895609570958095C2
:1069E000909530954095509521953F4F4F4F5F4F73
:1069F0006F4F7F4F8F4F9F4F08950F93083090F048
:106A0000982F872F762F652F542F432F322F222731
:106A10000850F4CF220F331F441F551F661F771FE6
:106A2000881F991F0A95B2F70F91089597FB10F8E8
:106A3000169400080F93083098F00850232F342F35
:106A4000452F562F672F782F892F902DF4CF05943F
:106A50009795879577956795579547953795279596
:106A60000A95AAF70F9108952A0D3B1D4C1D5D1D37
:106A70006E1D7F1D801F911F08952A153B054C0533
:106A80005D056E057F058007910708950024A7FD29
:106A900000942A17300540055005600570058005F3
:106AA00090050895AA1BBB1B51E107C0AA1FBB1F7D
:106AB000A617B70710F0A61BB70B881F991F5A958A
:106AC000A9F780959095BC01CD0108950F931F9370
:106AD000CF93DF938230910510F482E090E0E09153
:106AE0000D07F0910E0720E030E0A0E0B0E0309715
:106AF00019F1408151810281138148175907C8F06B
:106B00008417950769F4109731F012960C93129739
:106B100013961C9327C000930D0710930E0722C0F5
:106B20002115310519F04217530718F49A01BD01D8
:106B3000EF01DF01F801DBCF21153105F9F0281B4A
:106B4000390B2430310580F48A819B8161157105F0
:106B500021F0FB019383828304C090930E078093FE
:106B60000D07FE01329644C0FE01E20FF31F819330
:106B7000919322503109398328833AC020910B0721
:106B800030910C07232B41F42091B7013091B801CB
:106B900030930C0720930B072091B5013091B6017B
:106BA0002115310541F42DB73EB74091B9015091FF
:106BB000BA01241B350BE0910B07F0910C07E2178B
:106BC000F307A0F42E1B3F0B2817390778F0AC0110
:106BD0004E5F5F4F2417350748F04E0F5F1F5093ED
:106BE0000C0740930B078193919302C0E0E0F0E023
:106BF000CF01DF91CF911F910F910895CF93DF9334
:106C0000009709F481C0FC01329713821282A0918F
:106C10000D07B0910E07109781F420813181820F0A
:106C2000931F20910B0730910C072817390751F556
:106C3000F0930C07E0930B0767C0ED0120E030E014
:106C4000CE17DF0740F44A815B819E014115510553
:106C5000F1F0EA01F5CFD383C28340815181840FE3
:106C6000951FC817D90759F488819981840F951FFA
:106C70000296918380838A819B81938382832115ED
:106C8000310529F4F0930E07E0930D073DC0E901AB
:106C9000FB83EA8349915991C40FD51FEC17FD0777
:106CA00061F480819181840F951F0296E901998397
:106CB0008883828193819B838A83E0E0F0E012964F
:106CC0008D919C911397009719F0FD01DC01F7CF8E
:106CD0008D919C9111979D012E5F3F4F820F931FC5
:106CE00020910B0730910C072817390769F430976A
:106CF00029F410920E0710920D0702C0138212821F
:106D0000B0930C07A0930B07DF91CF910895A0E0FB
:106D1000B0E0EDE8F6E30C940532EC01009721F4C5
:106D2000CB010E946635B4C0FC01E60FF71F9C0141
:106D300022503109E217F30708F4A8C0D9010D91D8
:106D40001C91119706171707B0F00530110508F4CC
:106D50009BC0C80104978617970708F495C0025096
:106D60001109061B170B019311936D937C93CF01AF
:106D70000E94FE3589C05B01A01AB10A4C01800E49
:106D8000911EA0910D07B0910E07612C712CE12C82
:106D9000F12C109709F446C08D919C911197A8157C
:106DA000B905B1F56C0142E0C40ED11CCA14DB0474
:106DB00078F14C018A189B08640142E0C40ED11C92
:106DC0001296BC9012971396AC91B5E0CB16D104F5
:106DD00040F0B282A38391828082D9016D937C932B
:106DE00009C00E5F1F4F800F911FF90191838083AF
:106DF000EB2DFA2FE114F10431F0D7011396FC9337
:106E0000EE93129741C0F0930E07E0930D073CC03C
:106E10006816790608F43C017D0112960D90BC912C
:106E2000A02DB7CF80910B0790910C07881699067B
:106E3000E1F466167706C8F48091B5019091B60129
:106E4000009741F48DB79EB74091B9015091BA01B6
:106E5000841B950BE817F907C8F4F0930C07E0932F
:106E60000B07F901718360830FC0CB010E94663567
:106E70007C01009759F0A801BE010E945237CE0153
:106E80000E94FE35C70104C0CE0102C080E090E040
:106E9000CDB7DEB7EEE00C94213281E090E0F894BB
:106EA0000C946B37FB01DC0102C001900D92415044
:106EB0005040D8F70895FB01DC018D9101908019B5
:106EC0000110D9F3990B0895FB01DC0101900D929B
:106ED0000020E1F7089510E0C2E7D0E004C0FE0111
:106EE0000E94C4332196C337D107C9F7F894FFCF66
:106EF00020E0B201903B7E01D03F4401407D14016F
:106F000070E9D700406B9A0010936B00D0B1370046
:106F1000903A1C0079003C001F1115111D1D111F16
:106F20001F1115111515111F1F111D1D1D1D1D1FD1
:106F30001F1117111515111F1F1117111D1D111FDD
:106F40001F1515111D1D1D1F1F111D111D1D111FA9
:106F500070E9D70001320000000300CCF803009371
:106F600001BE01EA01FE01120226023A026C02BAD7
:106F700002E4020C0348035C03720388039D03A12F
:106F800003A403A803AC0340420F00B80B0000A801
:106F9000FDFFFF32454C000170E9D700C00E16021C
:106FA00001C0320A0300000F078000000204000342
:106FB00000011003020000030201000600040006A5
:106FC0000500200605040000000000C10C2E0C582E
:106FD0000C0E0D890C670C7B0C00000000C70D9A8D
:106FE0000DF60D6E0D920D7E0D6F0D00000000B0C0
:106FF0000F2E0CF60D2D0C550053534200436F72AB
:10700000722E504C4C2053693533353120200020EE
:10701000436F72726563742E2042464F2D312000FB
:1070200020436F72726563742E2042464F2D3220CA
:10703000002020202020434C4B202D2032202020D7
:1070400020004F6666004F6E200020202020204345
:107050004C4B202D20312020202000436F72722EB7
:1070600046696C7465722073697A6500487A2020DD
:107070002020200020436F72722E205368696674AE
:107080002043572000436F72722E20535F4C4556A9
:10709000454C2D3F00535752202020202020503DAA
:1070A00030572020202020005357523D0020503DD3
:1070B000005720202000FFFFFFFFFFFFFFFF072BEF
:1070C000363000FFFFFFFFFFFFFFFF072B353500C6
:1070D000FFFFFFFFFFFFFFFF072B353000FFFFFF24
:1070E000FFFFFFFFFF072B343500FFFFFFFFFFFF10
:1070F000FFFF072B343000FFFFFFFFFFFFFFFF07FD
:107100002B333500FFFFFFFFFFFFFFFF072B33305F
:1071100000FFFFFFFFFFFFFFFF072B323500FFFFE0
:10712000FFFFFFFFFFFF072B323000FFFFFFFFFFD6
:10713000FFFFFF072B313500FFFFFFFFFFFFFFFFC2
:10714000072B313000FFFFFFFFFFFFFFFF072B354D
:107150002000FFFFFFFFFFFFFFFF0720202000FFB1
:10716000FFFFFFFFFFFF062020202000FFFFFFFFA3
:10717000FFFF05202020202000FFFFFFFFFF04204D
:10718000202020202000FFFFFFFF032020202020C0
:10719000202000FFFFFF02202020202020202000B0
:1071A000FFFF0120202020202020202000FFFF20A2
:1071B00020202020202020202000FF202020202010
:1071C00020202020202000202020202020202020DF
:1071D000202020004C5342004C00555342004641B1
:1071E000003B00202050494E204130203D200030FF
:1071F0002042616C6C203D204F46462056464F2071
:1072000000332042616C6C3D20302E38206D6B566F
:107210002000362042616C6C3D2036206D6B56207C
:10722000202000392042616C6C3D203530206D6B90
:1072300056202000392B323064423D20353030203A
:107240006D6B562000392B343064423D2035303090
:1072500030206D6B5600392B363064423D2035307E
:107260003030306D6B560031487A20003130487A2A
:10727000003530487A003130304800353030480031
:10728000316B487A0031306B48003130306B00414F
:1072900075746F006E616E00696E66006F766600D1
:00000001FF
